:100000000C94890B0C94C4400C94E9400C94A60BFE
:100010000C94A60B0C94A60B0C94F3400C94A60B1A
:100020000C94A60B0C94FD400C94A60B0C94A60B00
:100030000C94A60B0C94A60B0C94A60B0C94A60B7C
:100040000C9481410C94A60B0C94A60B0C94A60B5B
:100050000C94A7410C94CE410C94FD410C94A60B3A
:100060000C94A60B0C94A60B0C94A60B0C94A60B4C
:100070000C94A60B0C94A60B0C94A60B312E3238C4
:100080002E30320034059A024C01A500520029009E
:100090001B00171515151515170012121212121242
:1000A000120017111117141417001711111711113D
:1000B0001700151515171111110017141417111128
:1000C0001700171414171515170000000000000082
:1000D000000092009A00A200AA00B200BA00C2007A
:1000E000CA004845414400474554202F005245422C
:1000F0004F4F540D0A0052455345540D0A004A4AC9
:1001000059004750530054532D4E545030315F58CE
:100110005858585858006E74702E6A73742E6D6655
:100120006565642E61642E6A70003030302E303088
:10013000302E3030302E303030003030302E3030F5
:10014000302E3030302E303030003030302E3030E5
:10015000302E3030302E3030300016012A013A0176
:100160004A0170079007B007D00730313233343579
:100170003637383941424344454600485454502F9D
:10018000312E312032303020485454500D0A436F04
:100190006E6E656374696F6E3A20636C6F73650D84
:1001A0000A436F6E74656E742D547970653A2074CD
:1001B0006578742F68746D6C0D0A43616368652DF2
:1001C000436F6E74726F6C3A206E6F2D636163685B
:1001D000650D0A436F6E74656E742D4C616E6775A4
:1001E0006167653A20656E0D0A0D0A004854545047
:1001F0002F312E3120323030204F4B0D0A436F6E9D
:100200006E656374696F6E3A20636C6F73650D0A77
:10021000436F6E74656E742D547970653A20746501
:1002200078742F68746D6C0D0A43616368652D43A3
:100230006F6E74726F6C3A206E6F2D6361636865C8
:100240000D0A436F6E74656E742D4C616E67756137
:1002500067653A20656E0D0A0D0A3C21444F4354F0
:100260005950452048544D4C205055424C4943204C
:10027000222D2F2F5733432F2F4454442048544DC1
:100280004C20342E3031205472616E736974696F62
:100290006E616C2F2F454E222022687474703A2FA5
:1002A0002F7777772E77332E6F72672F54522F6800
:1002B000746D6C342F6C6F6F73652E647464223EA2
:1002C0003C48544D4C3E3C484541443E3C544954C6
:1002D0004C453E54532D4E54502D53455256455285
:1002E0002053455455503C2F5449544C453E3C2FC7
:1002F000484541443E3C424F4459204247434F4CBD
:100300004F523D22234646464646464646223E3CFE
:1003100043454E5445523E3C423E00223E3C2F4611
:100320004F524D3E3C42523E3C464F4E5420434F6E
:100330004C4F523D22475245454E223E56414C5568
:10034000452053415645443C2F464F4E543E3C4277
:10035000523E00223E3C42523E3C42523E3C494EBE
:1003600050555420545950453D225355424D4954FF
:10037000222056414C55453D224150504C59223E79
:100380003C2F464F524D3E004950004E4D004757BE
:1003900000444E0042430088038B038E0391039474
:1003A000032000240028002C00C0006401A8C00025
:1003B000FFFFFF0101A8C00101A8C0FF01A8C049BB
:1003C000502041444452455353005355424E4554E6
:1003D000204D41534B004741544557415900444E2D
:1003E00053205345525645520041444452455353BD
:1003F00000BF03CA03D603DE03E9034E31004E32C9
:10040000004E33004E3400FB03FE0301040404538A
:1004100045525645523100534552564552320053CB
:100420004552564552330053455256455234000FFB
:100430000417041F042704400060008000A000008F
:10044000504F574552204F4E0045585445524E414B
:100450004C2052455345540042524F574E204F5561
:1004600054205245534554005741544348444F4744
:100470002054494D455220524553455400454E4362
:1004800032384A3630205245434549564520455278
:10049000524F52004152502052455155455354201D
:1004A00054494D454F5554204552524F52004943EF
:1004B0004D50205041434B455420434845434B2029
:1004C00053554D204552524F5200544350205041F5
:1004D000434B455420434845434B2053554D2045FD
:1004E00052524F5200554450205041434B455420E6
:1004F000434845434B2053554D204552524F5200DF
:1005000049434D50204D45535341474500444843CE
:10051000502052454345495645204E414B285245AF
:100520005452592900444843502052454E455741A2
:100530004C205354415445004448435020524542B6
:10054000494E4420535441544500444843502045AB
:10055000585049524544205354415445004448435F
:10056000502052454345495645205041434B455440
:10057000204552524F52004E425420524543454965
:100580005645204552524F52004E425420464F523B
:100590004D4154204552524F52004E42542050413A
:1005A000434B4554204552524F52004E4254205422
:1005B000494D45204F5554285345525645523129EF
:1005C000004E42542054494D45204F555428534520
:1005D000525645523229004E42542054494D45202E
:1005E0004F5554285345525645523329004E4254D4
:1005F0002054494D45204F55542853455256455295
:10060000342900444E532054494D45204F55542819
:10061000534552564552312900444E532054494DBA
:1006200045204F55542853455256455232290044CF
:100630004E532054494D45204F555428534552564A
:100640004552332900444E532054494D45204F55BF
:1006500054285345525645523429004E5450205583
:100660004E53594E43524F4E495A4544004E5450F2
:100670002054494D45204F55542853455256455214
:100680003129004E54502054494D45204F5554288F
:100690005345525645523229004E54502054494D2C
:1006A00045204F5554285345525645523329004E44
:1006B00054502054494D45204F55542853455256C7
:1006C00045523429004E545020494C4C4547414C2A
:1006D00020534552564552205245504C59004E54D5
:1006E00050204C454150205345434F4E44204144F7
:1006F0004A5553540054494D4520494C4C454741B7
:100700004C00475053204E4D454120464F524D41DD
:1007100054204552524F52004E4D454120434845CA
:10072000434B53554D204552524F520054494D456D
:1007300020444154412052454345495645204552A5
:10074000524F5200554E53594E432054494D455532
:1007500050003F0440044904580468047D04940494
:10076000AE04CA04E50400050D05250538054A0553
:100770005D05770589059A05AB05C105D705ED052A
:10078000030619062F0645065B066D0683069906C5
:10079000AF06C506DE06F506020718072C07440754
:1007A0006E772E636769006E732E636769006E62F1
:1007B0002E63676900636C2E63676900656C2E6346
:1007C00067690073642E6367690066617669636FA9
:1007D00000A007A707AE07B507BC07C307CA0746AF
:1007E0004958204E4554574F524B20534554544975
:1007F0004E470054494D45205345525645522053CB
:10080000455454494E470054494D452050524F5687
:100810004944452053455454494E470054494D4599
:100820002042524F414443415354204C4F470045CE
:1008300056454E54204C4F470053595354454D2074
:10084000494E464F4D4154494F4E00DF07F30707CD
:10085000081C082F0839084E54502041444A55536B
:10086000544D454E54204D4F44450042524F414453
:10087000434153542041444A5553544D454E54200E
:100880004D4F4445004750532041444A5553544D21
:10089000454E54204D4F4445004A4A5920434C4F41
:1008A000434B2041444A5553544D454E54204D4FDF
:1008B00044450057086B08850899084E4F20414C65
:1008C00041524D2854494D452053594E43524F4EA5
:1008D000495A4544290054494D4520414C41524D07
:1008E000284E4F542053594E43524F4E495A454477
:1008F000290054494D4520554E41444A55535445CD
:10090000440054494D45204F5045524154494F4EA3
:100910002054494D454F555400555443204D4F44A4
:10092000452854494D452056414C494429005554C9
:1009300043205050534F5554204D4F44452854495F
:100940004D452056414C49442900475053205449B5
:100950004D45204E4F2056414C4944004E4F2054A7
:10096000494D4520494E50555400BB08D608F20861
:10097000020919092E094A095C0920485454502FCC
:10098000003C2F413E3C42523E003F223E003C4252
:10099000523E3C4120485245463D222E2F005453A2
:1009A0002D4E54502D5345525645523C2F423E3CFD
:1009B00042523E004243004954424C00223E3C42D7
:1009C000523E3C42523E494E54455256414C2853A9
:1009D00065632E2030206F72203E3635353334204B
:1009E00049676E6F7265293C42523E3C494E5055F4
:1009F0005420545950453D225445585422204E41CC
:100A00004D453D224954424C222053495A453D22EE
:100A10003822204D41584C454E4754483D223522FE
:100A20002056414C55453D22003530223E3C2F5446
:100A3000483E3C54482057494454483D22313530C3
:100A4000223E54494D453C2F54483E3C5448205783
:100A5000494454483D22313530223E414D4F554E98
:100A6000543C2F54483E3C54482057494454483D38
:100A700022313530223E4E4F54453C2F54483E3CA7
:100A80002F54523E003C2F54443E3C2F54523E00C3
:100A90003C2F54443E3C54443E26656D73703B00ED
:100AA0003C2F54443E3C54443E42432041444A552A
:100AB0005354006D732E007365632C006F7665725E
:100AC0002039686F7572732E00444953545249425D
:100AD0005554494F4E002D2D2D2D2D3C2F54443E65
:100AE0003C54443E003C2F54443E3C54443E00267B
:100AF000656D73703B003C2F54443E3C54443E00B3
:100B00003C545220414C49474E3D2243454E5445AA
:100B100052223E3C54443E004552525253540043EC
:100B20004C520050473D3100313530223E54494D42
:100B3000453C2F54483E3C54482057494454483D76
:100B400022353030223E4556454E543C2F54483EC7
:100B50003C2F54523E003C2F54443E3C2F54523EB6
:100B60000026656D73703B3C2F54443E3C54443E1C
:100B700026656D73703B002C44415441313A002C82
:100B8000434F44453A0028545950453A002C4E45AD
:100B900058543A002C434E543A00285354533A00C8
:100BA0003C2F54443E3C54443E002D2D2D2D2F2DE2
:100BB0002D2F2D2D202D2D3A2D2D3A2D2D003C544D
:100BC0005220414C49474E3D2243454E5445522206
:100BD0003E3C54443E003C2F5441424C453E3C4236
:100BE000523E004F5045524154494E472054494DC2
:100BF00045004D494E2E00484F555220004649525F
:100C00004D574152452056455253494F4E00454E8F
:100C10004332384A3630205245564953494F4E00E8
:100C20004D414320414444524553530054494D459E
:100C300020535441545553004F5045524154494F4D
:100C40004E204D4F4445004E455442494F53204E8F
:100C5000414D4500444E532053455256455200479E
:100C60004154455741592041444452455353005340
:100C700055424E4554204D41534B0049502041446C
:100C8000445245535300323030223E4954454D3C86
:100C90002F54483E3C54482057494454483D223341
:100CA0003030223E56414C55453C2F54483E3C2F57
:100CB00054523E003C2F54443E3C2F54523E003C84
:100CC0002F54443E3C54443E003C545220414C4935
:100CD000474E3D2243454E544552223E3C54443EED
:100CE00000222056414C55453D220022204D4158BE
:100CF0004C454E4754483D2200222053495A453D19
:100D000022003C42523E3C494E50555420545950CA
:100D1000453D225445585422204E414D453D220028
:100D2000223E3C42523E003C42523E3C2F43454E06
:100D30005445523E3C2F424F44593E3C2F48544D5F
:100D40004C3E003C42523E3C4120485245463D22EA
:100D50002E2F223E4D41494E204D454E553C2F41B0
:100D60003E3C42523E003C42523E003F45525252AF
:100D70005354223E4552524F52204F46463C2F413B
:100D80003E3C42523E0026656D73703B3C4120481C
:100D90005245463D22003F434C52223E4C4F472095
:100DA000434C4541523C2F413E003F50473D31228C
:100DB0003E5B325D3C2F413E26656D73703B3C418E
:100DC00020485245463D22003F50473D30223E5B81
:100DD000315D3C2F413E26656D73703B3C412048A0
:100DE0005245463D22003C2F5441424C453E3C4238
:100DF000523E3C4120485245463D22003C2F423E57
:100E00003C42523E3C42523E3C5441424C452042C0
:100E10004F524445523D2231223E3C54523E3C54B6
:100E2000482057494454483D220022204D4554480B
:100E30004F443D22474554003C2F423E3C42523EE7
:100E40003C464F524D20414354494F4E3D220053A2
:100E5000554E004D4F4E00545545005745440054E3
:100E60004855004652490053415400414955545594
:100E700050564E54532D4E54502D534552564552B4
:100E8000303100454E4332384A3630205245563ACA
:100E900000494E495449414C495A494E472E2E2E3D
:100EA00000494E495449414C495A4544004B455923
:100EB000494E50555420494C4C4547414C004D54E7
:100EC0004B3333333920494E49542E2E2E004341A3
:100ED0004C2052454D3A0044484350204449534128
:100EE000424C4544004448435020454E41424C4505
:100EF00044004E545020525820454E41424C4544E7
:100F0000004E54502052582044495341424C4544CD
:100F10000042524F414443415354204C4F47004FED
:100F20005045524154494E472054494D4500475081
:100F300053204D4F4445205245414459004A4A5997
:100F4000204D4F4445205245414459004655525585
:100F50004E4F20475053204D4F444500554E495663
:100F600020475053204D4F444500454E4332384AA8
:100F7000363020494E495445525200730E830E912B
:100F80000EA10EAD0EBE0ECE0ED70EE50EF20E0168
:100F90000F110F1F0F2E0F3D0F4C0F5C0F6A0F56D6
:100FA000657273696F6E00504C454153452043484C
:100FB00045434B204B455900504C45415345205229
:100FC00045534554004D41433A0044484350434E35
:100FD000543A004E42432052454D3A00574149543D
:100FE00020666F722054494D4520525800434F4EA1
:100FF0004E4543542054532D4A4A593032004348F9
:1010000045434B204349524355495400504C4541B8
:101010005345205741495400434845434B20434FD3
:101020004E4E4543544F52009F0FA70FB80FC50FA8
:10103000CA0FD30FDC0FED0FFE0F0C101810455820
:101040005049524544200020524542494E44200018
:1010500052454E4557414C2000494E46494E495451
:1010600059003E104710501059104A5354004B532A
:1010700054004343540055544300505354004844D3
:1010800054006A106E10721076107A107E102020B4
:101090002020202020202020202020202020005040
:1010A0004F574552204F4E0045585445524E414CE3
:1010B0002052455345540042524F574E204F5554ED
:1010C000205245534554005741544348444F47200C
:1010D000524553455400454E4320524356204552F5
:1010E000524F5200415250205245512054494D45D3
:1010F0004F55540049434D502053554D20455252B1
:101100004F52005443502053554D204552524F5298
:10111000005544502053554D204552524F520049DE
:10112000434D50204D4553534147452052435600AF
:10113000444843502052454345495645204E414B73
:1011400000444843502052454E4557414C004448C6
:10115000435020524542494E4400444843502045A4
:10116000585049524544004448435020504354206D
:101170004552524F52004E4254205243562045523F
:10118000524F52004E425420464F524D415420453A
:1011900052524F52004E4254205041434B4554202E
:1011A0004552524F52004E42542054494D454F55DE
:1011B00054284E6F3129004E42542054494D454F1A
:1011C0005554284E6F3229004E42542054494D4503
:1011D0004F5554284E6F3329004E42542054494DE8
:1011E000454F5554284E6F342900444E53205449DE
:1011F0004D454F5554284E6F312900444E532054CD
:10120000494D454F5554284E6F322900444E5320C6
:1012100054494D454F5554284E6F332900444E5381
:101220002054494D454F5554284E6F3429004E5493
:101230005020554E53594E43524F4E495A45004E39
:1012400054502054494D454F5554284E6F31290074
:101250004E54502054494D454F5554284E6F322915
:10126000004E54502054494D454F5554284E6F332D
:1012700029004E54502054494D454F5554284E6F27
:101280003429004E545020494C4C4547414C205283
:1012900045502E004E5450204C4541502041444A68
:1012A0005553540054494D4520494C4C4547414CF9
:1012B0000047505320464F524D4154204552524F03
:1012C00052004E4D45412043484B53554D20455209
:1012D000522E0054494D452044415441205243561A
:1012E00045525200554E53594E432054494D455591
:1012F00050008E109F10A810B710C710D610E41021
:10130000F410031111111F11301141114E115A1116
:101310006711761184119511A611B711C811D91151
:10132000EA11FB110C121D122E123F125012611203
:10133000721283129412A412B112C212D312E412C6
:101340002D2D2F2D2D202D2D3A2D2D3A2D2D0048D0
:101350004F55522020204D494E2E002A2A3A2A2A43
:101360003A2A2A002D2D3A2D2D3A2D2D0054494D83
:10137000450D0A00444154450D0A0061646A7573C5
:101380007465640076616C696400535455530D0AAA
:1013900000444353540D0A00524D43005A44410047
:1013A000504D544B3030312C3331342C33002450D9
:1013B0004D544B3331342C302C312C302C312C30DB
:1013C0002C302C302C302C302C302C302C302C303D
:1013D0002C302C302C302C302C312C302A32390D42
:1013E0000A0024504D544B3331342C302C312C30E6
:1013F0002C312C302C302C302C302C302C302C300C
:101400002C302C302C302C302C302C302C302C30FC
:101410002A32380D0A004649582049502041444498
:101420005245535300464958205355424E45542087
:101430004D41534B004649582044464C54204741A7
:1014400054455741590046495820444E532053456E
:10145000525645520044484350205553452F554E4F
:1014600055534500424C4F4144434153542041445D
:1014700044522E00424C4F41444341535420494E64
:1014800054564C0042434153542043414C20524552
:1014900043562E0054494D45205A4F4E4500475063
:1014A00053204E4F444154412054494D455200472A
:1014B000505320554E53594E432054494D455200E8
:1014C0004E4D45412053454E54454E5345003150F5
:1014D000505320494E5055542045444745004E54E2
:1014E000502052582054494D454F55540041444ACC
:1014F00055535420574944544800475053204241C3
:101500005544205241544500484F55522053595399
:1015100054454D005155495420544F204D41494E9A
:1015200000161425143514461455146414741484C8
:101530001494149E14AF14C014CE14DE14ED14FAD7
:1015400014081514154A5354285554432B393A306E
:101550003029004B5354285554432B393A30302905
:1015600000434354285554432B383A303029005512
:1015700054432855544320303A30302900505354B6
:10158000285554432D383A303029004844542855C2
:1015900054432D393A303029004515531561156FE4
:1015A000157D158B15907E0000907E0000807000E8
:1015B0000000000000808FFFFF7081FFFF4D544B43
:1015C0003333333928244750524D432900554E496F
:1015D000562E28244750524D432900554E49562E29
:1015E000282447505A44412900BD15CD15DB154626
:1015F000414C4C2045444745005249534520454401
:10160000474500EF15F91544495341424C45004503
:101610004E41424C450007160F1644495341424C77
:101620004500454E41424C45284E5450204D4F44B4
:101630004529001A162216203132303062707300AC
:1016400020323430306270730020343830306270B1
:1016500073002039363030627073003139323030E7
:10166000627073003338343030627073003537364F
:1016700030306270730037164016491652165B16EA
:1016800064166D16323420484F5552205359535426
:10169000454D00323820484F555220535953544538
:1016A0004D00333020484F55522053595354454D27
:1016B0000084169316A21657494454483A20202015
:1016C00020207365630054494D454F55543A2020FE
:1016D0002020206D7300544F55543A2020202020A4
:1016E00073656300544F55543A20202020207365C1
:1016F0006300494E54455256414C3A202020202048
:1017000073002F3138002D2D204D454E55202D2DA5
:10171000000011241FBECFEFD0E1DEBFCDBF12E02D
:10172000A0E0B1E0ECE4F7EC02C005900D92A83B1C
:10173000B107D9F71CE0A8EBB2E001C01D92A732B7
:10174000B107E1F70E94E50E0C94A4630C9400002D
:1017500080917B01882359F48091EB099091EC09E9
:1017600090930A0C8093090C81E080937B0108958B
:10177000A0E2B0E0EEEBFBE00C9439620E94721A3A
:1017800082E00E94BF4B01C0A895F999FDCF86E089
:1017900090E063E070E00E949F6301C0A895F99912
:1017A000FDCF8EE090E060E570E00E949F6301C095
:1017B000A895F999FDCF8CE090E06AE070E80E946E
:1017C0009F6301C0A895F999FDCF80E290E044E6BF
:1017D00051E068EA70EC0E94976301C0A895F999FE
:1017E000FDCF84E290E040E05FEF6FEF7FEF0E947B
:1017F000976301C0A895F999FDCF88E290E041E098
:1018000051E068EA70EC0E94976301C0A895F999CD
:10181000FDCF8CE290E041E051E068EA70EC0E947C
:101820009763CE01019666E071E00E94926201C06A
:10183000A895F999FDCFCE01019660E170E040E1F5
:1018400050E00E947F6301C0A895F999FDCF8E01F9
:101850000F5F1F4FC80166E171E00E949262C801EC
:1018600060E470E040E250E00E947F6301C0A89510
:10187000F999FDCF8E010F5F1F4FC8016AE271E039
:101880000E949262C80160E670E040E250E00E946F
:101890007F6301C0A895F999FDCF8E010F5F1F4F9F
:1018A000C8016AE371E00E949262C80160E870E0DA
:1018B00040E250E00E947F6301C0A895F999FDCFF6
:1018C0008E010F5F1F4FC8016AE471E00E949262AF
:1018D000C80160EA70E040E250E00E947F6301C00E
:1018E000A895F999FDCF80EC90E04FEF51E068EAC0
:1018F00070EC0E94976301C0A895F999FDCF84EC24
:1019000090E060E070E00E949F6301C0A895F999A3
:10191000FDCF86EC90E060ED77E00E949F6301C010
:10192000A895F999FDCF88EC90E068E873E10E94F2
:101930009F6301C0A895F999FDCF8CE390E068E022
:1019400070E00E949F6301C0A895F999FDCF8CECCF
:1019500090E060E070E00E949F6301C0A895F99953
:10196000FDCF80ED90E064EB70E00E949F6301C0CA
:10197000A895F999FDCF82ED90E064E873E00E94AC
:101980009F6301C0A895F999FDCF8EE390E065EAC9
:1019900073EC0E949F63A096E4E00C9455620E9451
:1019A000D71D83B180958F70873069F40E94B80B82
:1019B0000E94721A83E00E94BF4B82E00E94B24BE9
:1019C000A895FECFA895F999FDCF8EE390E00E94EF
:1019D0004563855A934C21F00E94B80B01C0A8952D
:1019E000F999FDCF86E090E00E9445639C0181500B
:1019F0008E3F08F025E020938B0401C0A895F9994B
:101A0000FDCF8EE090E00E94456390936305809344
:101A1000620501978E5F9F4F40F080E590E09093C4
:101A200063058093620501C0A895F999FDCF8CE00C
:101A300090E00E9445639C019F77909352088093A9
:101A40005108C90101978E5F9F4F50F084E1809348
:101A500054088CE390E0909352088093510810C092
:101A600037FF0CC08091E7099091E809019711F0C8
:101A700084E101C085E18093540802C010925408AB
:101A800080915408882309F040C080E290E044E649
:101A900051E068EA70EC0E94861C609329057093FF
:101AA0002A0580932B0590932C0584E290E040E07A
:101AB0005FEF6FEF7FEF0E94861C60932D057093A0
:101AC0002E0580932F059093300588E290E041E049
:101AD00051E068EA70EC0E94861C609331057093B7
:101AE000320580933305909334058CE290E041E019
:101AF00051E068EA70EC0E94861C6093DD097093E7
:101B0000DE098093DF099093E00980E190E06DECBD
:101B100079E046E051E00E94631C8091030166ED8C
:101B200079E00E94483C8091040168ED79E00E94D0
:101B3000483C809105016AED79E00E94483C80EDC7
:101B400090E00E9445632FEF8F3F920711F484EBE2
:101B500090E09093EA098093E90982ED90E00E9479
:101B600045634FEF8F3F940711F484E893E090931F
:101B7000EC098093EB0980E490E060E777E046E1D0
:101B800051E00E94401C80E690E060E977E04AE284
:101B900051E00E94401C80E890E060EB77E04AE36F
:101BA00051E00E94401C80EA90E060ED77E04AE45A
:101BB00051E00E94401C80EC90E04FEF51E068EA59
:101BC00070EC0E94861C6093F6077093F707809371
:101BD000F8079093F90701C0A895F999FDCF84EC17
:101BE00090E00E94456390931708809316088F5FDA
:101BF0009F4F31F4109217081092160801C0A89553
:101C0000F999FDCF86EC90E00E944563909315080A
:101C10008093140801978E5F9F4F40F080ED97E00E
:101C2000909315088093140801C0A895F999FDCFE9
:101C300088EC90E00E94456390931C0880931B08F9
:101C40008F5F9F4F31F488E893E190931C08809355
:101C50001B088091E409882311F015C0A895F99913
:101C6000FDCF8AEC90E00E94456397FD0CC080FF99
:101C70000AC08091E309887F8093E30981E0809323
:101C8000E40901C0A895F999FDCF8CE390E00E948A
:101C900045639C014FEF8F3F940711F428E030E03B
:101CA000422F47708091E309482B4093E30923FFBB
:101CB00003C048604093E309832F83708093FD093C
:101CC00001C0A895F999FDCF8CEC90E00E94456386
:101CD0008093F2098F3F21F41092F20901C0A89578
:101CE000F999FDCF8091F209E82FF0E0EE0FFF1F88
:101CF000EE0FFF1FEB55FA4E85919591A591B4918A
:101D00008093770190937801A0937901B0937A0141
:101D10000895EF92FF920F931F93E0901608F090B2
:101D2000170800E010E083E591E06DE171E00E94AA
:101D3000753FE61AF70A080B190BB701C8011F9186
:101D40000F91FF90EF900895EF92FF920F931F93E2
:101D5000E0901808F09019080027F7FC0095102F64
:101D600081E491E06DE171E00E94753FE61AF70AA7
:101D7000080B190BB701C8011F910F91FF90EF904D
:101D800008950F931F938C010E94673E00511040ED
:101D90006F717070060F171F1093190800931808C1
:101DA0000C33110534F48CE390E090931908809380
:101DB0001808A1E4B1E0EDE1F1E082E101900D92BB
:101DC0008150E1F71F910F910895ACE1B0E0EBEE87
:101DD000FEE00C942B62F8941092680081E08CBBBA
:101DE0001DBA89E88093640080E885BF85BF80BF05
:101DF0009FEF92B980E185B918B813E01BB991B98A
:101E000080EB84B98FE787B982EC8AB988E090E0EB
:101E10000E943F6360931D0870931E0880931F0803
:101E20009093200889B18073803129F4119882E061
:101E30008093E40905C0803239F412981093E409C4
:101E400087E080937C0103C010981092E40980E140
:101E50008CBD81E08DBD16BC92E094BD83E085BD54
:101E600027EC27BD90936E001092B2009093B000C3
:101E700084E08093B1002093B3009093700084B706
:101E800080FF04C081E00E94874F13C081FF02C021
:101E900082E007C082FF02C083E003C083FF09C065
:101EA00084E00E94874F81E090E09093E80980935E
:101EB000E70914BE8CE028E130E00FB6F894A8954D
:101EC000209360000FBE8093600078940E94F11A06
:101ED0000E94CF0C80E58CBD8091E409823059F4DA
:101EE00080918B04E82FF0E0EE0FFF1FEC57FF4FBF
:101EF0008591949104C0833089F485EA90E09093B1
:101F0000C5008093C40082E08093C00086E0809387
:101F1000C20088E98093C1008091C6005E9A80E18A
:101F200090E00E94441B0E941516882381F484E1EE
:101F300062EA7AE00E9444150E94721A81E10E94CE
:101F4000BF4B88E00E94B24B1798A895FECF0E9425
:101F5000EB180E94721A80E00E94BF4B80E00E9442
:101F6000B24B88E061E04CE750E00E94A31A0E9467
:101F70004B1B8C010CC0A8958091E409823019F4A8
:101F80000E94015304C0833011F40E94F1500E945A
:101F90004B1B801B910B805D974068F30E94721A67
:101FA0008091E409833031F48EE00E94BF4B87E0DA
:101FB0000E94B24B8091E409823081F48091E30960
:101FC00090E087709070892B49F485E00E94BF4BA8
:101FD00089E00E94B24B81E00E94905280915408A7
:101FE0008823F1F081E090E09093560880935508A3
:101FF000A8E0B1E0EDE1F1E082E101900D928150C5
:10200000E1F780915408843119F40E94AB2803C091
:1020100086E10E948929882339F00E94874F04C0F5
:1020200010925608109255089091E409923049F4A4
:102030008091E30983FF02C083E006C090936900AA
:1020400005C0933031F482E08093690081E08CBB5D
:102050008DBB1092E8091092E7090E944B1B9C8FE0
:102060008B8FA8950E948422823019F40E94F02060
:1020700009C0833019F40E94642704C0843041F5FC
:102080000E94D124182F0E949E16112309F18091DD
:10209000E4098823D1F4163091F48091F309882360
:1020A000A1F0A1E4B1E0EDE1F1E082E101900D9257
:1020B0008150E1F71092CA091092F30906C01B3152
:1020C00021F480E490E00E94C10E812F0E94874F8E
:1020D0008091E409823019F40E94015304C08330D6
:1020E00011F40E94F150F8944090040C5090050CAB
:1020F0001092050C1092040C2090070C3090080CE4
:102100001092080C1092070C789431E04316510499
:1021100009F045C2F8948091000C9091010CA091B7
:10212000020CB091030C89839A83AB83BC837894AF
:10213000CE0101960E948A1E009729F480EC8093BC
:10214000060181E088C0DE011996FC0182E1019060
:102150000D928150E1F769857A854B855C852D85E7
:102160003E85809106018034F1F48091110C882322
:10217000A9F4232B99F4452B89F4672B79F48981F1
:102180009A81AB81BC810197A109B10989839A83A6
:10219000AB83BC8392E09093110C35C08091110CFD
:1021A000823089F52DC0803871F58091110C88231B
:1021B00051F52731310539F54B33510521F56B3395
:1021C000710509F589819A81AB81BC810196A11DB8
:1021D000B11D89839A83AB83BC838091000C90915D
:1021E000010CA091020CB091030C0196A11DB11D30
:1021F0008093000C9093010CA093020CB093030CFD
:1022000081E08093110C89819A81AB81BC812091FE
:102210007701309178014091790150917A01820FD4
:10222000931FA41FB51F89839A83AB83BC83CE0100
:1022300001960E948A1EADE1B1E0FC0182E10190AD
:102240000D928150E1F78091110C813039F4109298
:1022500006011092110C80937C010AC08091110C30
:10226000823031F4ACE3B0E0B0931E01A0931D01C5
:102270000E94E31E0E94B6300E948C2A80911608AC
:1022800090911708892B61F18091F4099091F509DB
:102290000197E1F40E94890E3B014C0116161706C6
:1022A000180619064CF10E949833882311F00E94F9
:1022B000874FA3E5B1E0EDE1F1E082E101900D92FD
:1022C0008150E1F782E00E941E5016C0A3E5B1E004
:1022D000EDE1F1E082E101900D928150E1F709C05A
:1022E000A3E5B1E0EDE1F1E082E101900D928150D2
:1022F000E1F76624772443018091F309882321F0D4
:10230000EE24FF2487018AC08091E4098823C1F468
:102310000E94A40E7B018C011616170618061906DA
:102320000CF46BC08091290590912A05A0912B0592
:10233000B0912C050097A105B10509F45EC011C04C
:10234000833099F48091130C882309F053C00E94C4
:10235000A40E7B018C0116161706180619060CF43C
:102360004CC081E08093F30948C0823009F042C03C
:102370002091E9093091EA0921153105D9F08091C0
:102380000B0C90910C0C019690930C0C80930B0C01
:1023900080910B0C90910C0C8217930778F0B7E0AA
:1023A000B0937C0180917B01843041F023E0209345
:1023B0007B0104C010920C0C10920B0C80917B01DD
:1023C0008130C1F48091EB099091EC09892B91F057
:1023D0008091090C90910A0C019790930A0C8093BC
:1023E000090C8091090C90910A0C892B19F432E0A8
:1023F00030937B01EE24FF2487018091120C882307
:1024000031F08091120C81508093120C07C08091A2
:102410007C01853019F484E080937C018091F1097E
:102420008F5F8093F1098C33A9F41092F1098091A8
:10243000ED099091EE09A091EF09B091F009019694
:10244000A11DB11D8093ED099093EE09A093EF09B2
:10245000B093F0092091000C3091010C4091020CD6
:102460005091030C8091770190917801A0917901AE
:10247000B0917A01280F391F4A1F5B1F29833A83C5
:102480004B835C838091FD09813061F42054384393
:10249000404050402D833E834F83588754E0A52E03
:1024A000B12C10C0823019F0AA24BB240BC02056D6
:1024B0003445404050402D833E834F83588746E04B
:1024C000A42EB12CCE0105960E948A1EDE0119961B
:1024D000FC0182E101900D928150E1F7CF84D88810
:1024E000CE0101960E948A1EFC01A114B104D1F014
:1024F00086819781C816D906A9F0D88ACF869F0110
:10250000AE01475F5F4F82E1DA010D90AD01D90165
:102510000D929D018150C1F7848195818A0D9B1D8B
:1025200095838483AFE2B1E082E101900D92815006
:10253000E1F78091E109882319F40E94AC4D2FC086
:10254000843019F40E94884C2AC0853021F580918E
:10255000E409823039F0813029F08091F309882331
:1025600009F4E5C180E00E94AB4B80911608909180
:102570001708892B61F08091F4099091F509019772
:1025800031F481E0B401A3010E943E4C08C081E017
:102590000E94AB4B04C0863011F40E94CC4BB1E0DA
:1025A0002B16310409F04DC08091E409882321F0F5
:1025B000813031F40E941E5010927C0110927B01F8
:1025C0008091E409882311F0833031F58091180857
:1025D000909119082091FC09213019F4959587955F
:1025E0000BC0223049F4880F991F24E081309207F4
:1025F0001CF080E094E005C08034910514F480E480
:1026000090E00E94C10EA1E4B1E0EDE1F1E082E1D1
:1026100001900D928150E1F71092F30980911B0116
:1026200090911C01019769F410921C0110921B01FA
:10263000A3E5B1E0EDE1F1E082E101900D9281507E
:10264000E1F78091CA098823D9F00E940731182F39
:102650008823E1F080518B3058F4A1E4B1E0EDE142
:10266000F1E082E101900D928150E1F70E94583231
:102670001092CA091092F309812F0E94874F06C059
:102680001092C9091092CC091092CB098091E409EB
:10269000823080F40E94F232182F882359F0109271
:1026A000CA091092F30980E490E00E94C10E812FC4
:1026B0000E94874F31E043165104F1F480913E05AA
:1026C000882359F080914F05815080934F058823CE
:1026D00021F480E090E00E949324809150058823AB
:1026E00059F080916105815080936105882321F420
:1026F00081E090E00E9493248091E5099091E609A1
:10270000019711F40E94874E1092E6091092E50994
:102710000E944B1BAB8DBC8D8A1B9B0B409708F412
:10272000A4C00E944B1B9C8F8B8F0E94CD1B0E94CC
:10273000DC1B882309F499C0179A9091E109843130
:1027400041F48091E209882309F08FC00E948759E3
:102750005AC0813149F49F5F80911A01891708F0AE
:10276000ECC09091E209E9C0823149F48091E2091C
:10277000981719F490911A01E0C09150DEC083318E
:10278000D1F48091E209882339F427E02093E2090B
:1027900036E130931A012AC0873039F487E18093FB
:1027A000E20996E290931A0128C01092E209A6E08D
:1027B000A0931A012DC0863189F48091F40990917B
:1027C000F509019709F051C00E949833882311F050
:1027D0000E94874F82E00E941E5047C0883179F4E2
:1027E0008091E209873021F40E94714F97E0A5C0E3
:1027F000873109F0A2C00E947C4F97E19EC08F30C4
:1028000049F40E94F11A1092E209B6E0B0931A015D
:1028100090E093C0803149F58091E409823088F4DA
:102820008091F309882309F58091290590912A0563
:10283000A0912B05B0912C050097A105B105A9F039
:1028400002C0833091F481E08093F3090EC0892F98
:1028500087500E94C84C09C0873129F4892F8751BD
:102860000E94394D02C00E94874E80917B018823CF
:1028700021F080917B01813091F481E090E0909390
:10288000F5098093F4098091E4098250823028F49C
:102890001092060181E08093070115981EC0809177
:1028A0007B01833029F424E020937B0185E208C07A
:1028B00080917B01823031F434E030937B0186E2F9
:1028C0000E94874F1092F5091092F40980EC8093D2
:1028D000060190E190930701159A80911608909156
:1028E0001708892B41F08091F4099091F50901971F
:1028F00011F4149801C0149A80915408882371F03F
:102900008091290590912A05A0912B05B0912C0565
:102910000097A105B10511F0139801C0139A0E9408
:102920004E16813011F416989CCB169A9ACB80E003
:10293000B801A7010E943E4C18CE9093E109809106
:10294000E209873009F088CF82CF8EBD0DB407FE33
:10295000FDCF08952C988EBD0DB407FEFDCF1EBC93
:102960000DB407FEFDCF8EB52C9A08952C988EBD20
:102970000DB407FEFDCF1EBC0DB407FEFDCF8EB516
:102980001EBC0DB407FEFDCF8EB52C9A08952C9871
:10299000805C8EBD0DB407FEFDCF6EBD0DB407FE8D
:1029A000FDCF2C9A08950F931F93182F0E94AA14FD
:1029B000082F812F8F5F0E94AA14982F802F1F91BC
:1029C0000F9108950F931F93182F0E94B614082F8C
:1029D000812F8F5F0E94B614982F802F1F910F9127
:1029E00008950F931F93182F072F0E94C714812F4C
:1029F0008F5F602F0E94C7141F910F9108952C982C
:102A000080588EBD0DB407FEFDCF6EBD0DB407FE20
:102A1000FDCF2C9A08952C9880568EBD0DB407FEDC
:102A2000FDCF6EBD0DB407FEFDCF2C9A08951F9308
:102A3000182F8FE163E00E940B158FE1612F0E9438
:102A4000FF141F9108951F93182F82E00E941715FD
:102A500084E1612F0E94C71482E161E00E94C714E3
:102A600083E00E9417158AE00E94B61480FDFBCF18
:102A700082E00E94171582E160E00E94C71488E19D
:102A80000E94E2141F910895FF920F931F93F82E56
:102A90008B0182E00E94171584E16F2D0E94C714FC
:102AA00086E1B8010E94F11483E00E9417158AE0C4
:102AB0000E94B61480FDFBCF1F910F91FF900895E7
:102AC0002C988AE38EBD0DB407FEFDCF1EBC0DB45D
:102AD00007FEFDCF8EB52C9A08952C988AE38EBD03
:102AE0000DB407FEFDCF1EBC0DB407FEFDCF9EB595
:102AF0001EBC0DB407FEFDCF8EB52C9A08952C9800
:102B00008AE38EBD0DB407FEFDCF1EBC0DB407FEDB
:102B1000FDCF9EB51EBC0DB407FEFDCF8EB51EBC0D
:102B20000DB407FEFDCF7EB51EBC0DB407FEFDCF74
:102B30006EB52C9A0895FC012C988AE38EBD0DB4D5
:102B400007FEFDCF20E030E008C01EBC0DB407FE3C
:102B5000FDCF8EB581932F5F3F4F26173707A8F320
:102B60002C9A0895982F2C988AE78EBD0DB407FEF5
:102B7000FDCF9EBD0DB407FEFDCF2C9A0895282FE2
:102B80002C988AE78EBD0DB407FEFDCF9EBD0DB417
:102B900007FEFDCF2EBD0DB407FEFDCF2C9A089584
:102BA000282F2C988AE78EBD0DB407FEFDCF9EBD61
:102BB0000DB407FEFDCF2EBD0DB407FEFDCF7EBDCB
:102BC0000DB407FEFDCF6EBD0DB407FEFDCF2C9AF0
:102BD0000895FC012C988AE78EBD0DB407FEFDCF49
:102BE00020E030E008C080818EBD0DB407FEFDCF2F
:102BF0002F5F3F4F319626173707A8F32C9ACB014A
:102C00000895282F2C988AE78EBD0DB407FEFDCFBE
:102C100080E090E005C02EBD0DB407FEFDCF01960B
:102C200086179707C0F32C9A08958FE160E00E9401
:102C3000C71480E160E070E00E94F11482E16FEF60
:102C40007FE10E94F1148AE06FEF7FE10E94F114AE
:102C500083E00E94171587E067E00E94C71487E0B1
:102C60000E94AA1480FDFBCF87E062E00E940B1552
:102C70008FE160E30E94FF148FE10E94AA1485FD9A
:102C8000FBCF80E00E94171586E10E94D31420E05C
:102C90008750984F09F421E0822F089581E00E9427
:102CA00023159695879596958795817008958FE160
:102CB0000E94AA148095881F8827881F0895EF9284
:102CC000FF920F931F938C0180E00E94171580E004
:102CD0000E94E214F82EE92E6091930470919404FE
:102CE0006A5F7F4F600F711F89E1683D780710F0C0
:102CF000685D794180E00E94F1148F2D9E2D1F9117
:102D00000F91FF90EF900895EF92FF920F931F9312
:102D10008C0180E00E94171582E00E94E214F82ED8
:102D2000E92E0752164E82E0B8010E94F1148F2D51
:102D30009E2D1F910F91FF90EF9008950F931F9379
:102D400000919504109196040150104080E00E947B
:102D500017158EE160E40E94FF14B80189E1083D77
:102D6000180710F067ED79E18CE00E94F1141F91D3
:102D70000F9108951F93CF93DF9381E00E94171561
:102D800089E10E94AA14182F80E00E9417158EE096
:102D90000E94AA14C82FD0E081E00E94171589E193
:102DA0000E94AA14181779F78CE00E94D3149F711F
:102DB0008C179D0720F49C012952364E09C0C81774
:102DC000D90719F427ED39E105C09C0121503040A5
:102DD0002C1B3D0BC901DF91CF911F910895A7E0F6
:102DE000B0E0E5EFF6E10C9433628C01E0909804DA
:102DF000F0909904E80EF91E82E0B8010E94F114E7
:102E000080E00E94B21584E0B8010E94F11486E0CF
:102E1000B7010E94F1148FE160E80E94FF148FE176
:102E200060E80E940B158CE16AE00E940B158FE1AF
:102E300068E00E94FF14809197048550823008F06A
:102E400068C000E010E08CE10E94AA148A7031F49E
:102E50000F5F1F4F83E0083E1807A9F78CE10E941F
:102E6000AA1481FD05C083E0083E180708F451C08C
:102E70008FE168E00E940B1580E00E94E2145C0183
:102E800086E00E94E2146C010894C11CD11C80E011
:102E9000B6010E94F1148E010F5F1F4FC80167E059
:102EA00070E00E949B15EE24F02E012F8CE10E9411
:102EB000AA1481FF2AC08C8185FF27C08FE160E8BA
:102EC0000E94FF148FE160E80E940B158CE16AE01C
:102ED0000E940B158FE168E00E94FF148CE10E94B4
:102EE000AA148A70D9F38FE168E00E940B1580E084
:102EF000B6010E94F1148F2D902F67E070E00E94C0
:102F00009B15E39480E1E81689F680E0B5010E9404
:102F1000F1142796EAE00C944F62A0E0B0E0E3E9F8
:102F2000F7E10C943462B82E282F392F6901EE2472
:102F3000FF24870111C00E946015D82F0E946015E0
:102F4000C82FCE01A0E0B0E0E80EF91E0A1F1B1F3B
:102F50008EEF9FEFC80ED91E92E0C916D10458F724
:102F6000C701D8019C01AD01B0FE0BC00E946015E5
:102F7000D82FC0E09E0140E050E02E0D3F1D401FC5
:102F8000511F203080E0380781E0480780E0580773
:102F9000A0F0CA0140E050E0A0E0B0E0280F391FE7
:102FA0004A1F5B1F203090E0390791E0490790E00D
:102FB000590718F0C90101969C01C901CDB7DEB7C8
:102FC000E9E00C9450620F931F938B010E945F16EF
:102FD000C8010E948D179C0120953095C9011F9151
:102FE0000F910895EF92FF920F931F938C017B0135
:102FF00080E00E9417150752164E80E0B8010E942B
:10300000F114C7010E948D179C0120953095C901CC
:103010001F910F91FF90EF900895A0E0B0E0E3E1E1
:10302000F8E10C9435626C017B018A014115510570
:1030300009F444C04130510551F40E945F16C701A4
:103040000E9484160E9460150E94B21537C080E06D
:103050000E941715C0919304D09194042696CC0D2C
:10306000DD1D89E1C83DD80710F0C85DD94180E178
:10307000BE010E94F114B801615070406C0F7D1FB9
:1030800099E1683D790710F0685D794182E10E941D
:10309000F11489ED99E1E80EF91E84E1B7010E946F
:1030A000F1148FE160E10E940B158FE160E20E9454
:1030B000FF148FE10E94AA1485FDFBCFCDB7DEB7C8
:1030C000E8E00C9451628FE164E00E940B158DE101
:1030D0000E94AA1482FDFBCF8FE10E94AA1487FDF3
:1030E000FBCF8EE160E20E94FF1408951F93182F1A
:1030F00083E00E94171585E1612F0E94C7141F917C
:10310000089583E00E94171585E10E94AA1408958E
:10311000FC012C988AE38EBD0DB407FEFDCF20E0A4
:1031200030E00AC01EBC0DB407FEFDCF8EB5819302
:103130002F5F3F4F841719F02617370798F3108237
:103140002C9AC90108950F931F93CF93DF938C019D
:10315000C0E0D0E003C00E9460152196C017D107DF
:10316000D0F3DF91CF911F910F910895CF93DF930B
:10317000EC010E949962AC012C988AE78EBD0DB4D7
:1031800007FEFDCF20E030E00AC0FE01E20FF31F92
:10319000E491EEBD0DB407FEFDCF2F5F3F4F241726
:1031A000350798F32C9ACA01DF91CF9108958EE1EB
:1031B00060E20E940B1580E190E00E94441B8DE1CB
:1031C0000E94AA1483FDFBCF80FFF9CF8FE164E05A
:1031D0000E94FF1408951F938EE160E20E940B1578
:1031E00080E190E00E94441B5E9880E190E00E94A4
:1031F000441B5E9A80E190E00E94441B1FEF2C98D4
:103200001EBD0DB407FEFDCF2C9A80E190E00E9418
:10321000441B8DE10E94AA1483FDF1CF80FFEFCF04
:103220008FE160EC0E94C7148EE160E80E94C71431
:1032300088E060E070E00E94F1148CE067ED79E1D5
:103240000E94F1148AE067ED79E10E94F11484E0B4
:1032500068ED79E10E94F11481E00E94171588E180
:1032600061EA0E94C71482E00E94171580E06DE0B9
:103270000E94C71481E060E00E94C71482E062E30C
:103280000E94C7148AE06EEE75E00E94F11486E099
:1032900062E17CE00E94F11484E062E10E94C714C4
:1032A00083E060E40E94C71489E06FE30E94C714C2
:1032B00083E00E94171585E160E00E94C71484E056
:1032C000609100010E94C71485E0609101010E9495
:1032D000C71482E0609102010E94C71483E06091EC
:1032E00003010E94C71480E0609104010E94C7148A
:1032F00081E0609105010E94C71482E10E94AA1436
:103300008F718093970480E060E070E00E94441524
:1033100080E160E071E00E94441584E162E774E0BE
:103320000E94441580E00E9417158FE164E00E941E
:10333000C7141F910895CF93DF93EC0181E00E94A1
:10334000171589E10E94AA14882321F40E941715F9
:1033500080E044C080E00E94171560919504709150
:10336000960480E00E94F114809195049091960457
:1033700090939404809393048DE894E066E070E069
:103380000E949B1580918E048F7180938E04809192
:1033900090048F718093900420918D0430918E045D
:1033A000309396042093950480918F04909190041B
:1033B0008F5E954080F489E1283D380760F420FD58
:1033C0000AC08091920487FD06C08091910484FD1B
:1033D00002C087FD06C00E94EB1882E0DF91CF910A
:1033E0000895F8948091000C9091010CA091020C2A
:1033F000B091030C8093060890930708A0930808E7
:10340000B09309088091FE0B9091FF0B90930F08E9
:1034100080930E087894CE016EE070E00E949B15B8
:1034200081E0DCCF98B18F70907F892B88B90895A7
:10343000469898B18F70907F892B88B90000449A84
:1034400083E090E00E94441B449808951F93182F36
:1034500088B1912F92959F70807F982B98B9449A4C
:1034600083E090E00E94441B449888B11F70807FE5
:10347000812B88B9449A83E090E00E94441B4498D1
:103480001F910895469A0E94261A089546980E9410
:10349000261A08950E94421A81E090E00E94441B7F
:1034A0000895CF93DF93EC0103C021960E944A1A3E
:1034B00088818823D1F7DF91CF91089580E10E9420
:1034C000461A81E090E00E94441B0895882311F47D
:1034D0008CE001C08EE00E94461A81E090E00E94DC
:1034E000441B089581E00E94461A89E190E00E9401
:1034F000441B0895662349F0613011F4805C05C0D7
:10350000623011F48C5E01C08C5A80680E94461AA9
:1035100081E090E00E94441B08950F931F93042FB5
:103520000E947A1A10E004C080E20E944A1A1F5FCB
:103530001017D4F31F910F910895682F80E040E198
:103540000E948D1A0895CF93DF93EA010E947A1AA0
:1035500003C00E944A1A2196FE0184918823C9F76C
:10356000DF91CF9108950F931F938A010E947A1AD9
:10357000C8010E94511A1F910F9108951F93142F93
:103580000E947A1A812F0E94421A81E090E00E94E4
:10359000441B1F9108950F931F93CF93DF938B01CB
:1035A000880F880F880F887380640E94461AC0E0D5
:1035B000D0E081E090E00E94441B81E090E00E9416
:1035C000441BF801EC0FFD1FE4918E2F0E94421A5C
:1035D0002196C830D10569F7DF91CF911F910F91E6
:1035E00008951F93CF93DF9388E290E00E94531BCE
:1035F00083E00E94181A82E490E00E94441B83E05A
:103600000E94181A81E090E00E94441B83E00E940F
:10361000181A81E090E00E94441B82E00E94181A70
:1036200081E090E00E94441B88E20E94461A81E0FB
:1036300090E00E94441B88E00E94461A81E090E0DE
:103640000E94441B81E00E94461A89E190E00E949A
:10365000441B86E00E94461A81E090E00E94441BD1
:103660008CE00E94461AC2EDD0E010E0FE016591A8
:103670007491812F0E94CB1A1F5F22961830B1F7E8
:10368000DF91CF911F91089528EC00002A95E9F76A
:103690000197D1F70895F8942091B8023091B902BA
:1036A0007894C9010895AC01F8942091B802309142
:1036B000B902789401C0A895F8948091B8029091CD
:1036C000B9027894821B930B84179507A0F3089591
:1036D000DC01F8947894809105048823A1F0F89493
:1036E000E0910304F0E0ED5FFC4F80818C938091CA
:1036F00003048F5F809303048091050481508093BD
:103700000504789481E00895A1E0B0E0EAE8FBE1E7
:103710000C9439628E010F5F1F4F01C0A895C8013C
:103720000E94681B8130D1F32196E4E00C9455622D
:10373000A1E0B0E0EEE9FBE10C943B62CE01019622
:103740000E94681B882321F1909186049F3740F0E6
:1037500010928A04109289041092860482E019C0A3
:103760008981E92FF0E0EA5FFB4F8083E92FEF5F6B
:10377000E09386048A3061F4F0E0EA5FFB4F108248
:103780001092860410928A041092890481E001C08C
:1037900080E02196E2E00C9457629091BE0283B1E2
:1037A000EAEBF2E0E90FF11D80958F7080839F5F57
:1037B00093709093BE0208959091BB028091BA02DB
:1037C00098238091BC0298238091BD02982341F1F7
:1037D000983011F494E11DC0943011F493E119C0B4
:1037E000923011F492E115C0913011F491E111C0C1
:1037F0009C3011F498E10DC0933011F49FE009C0A2
:10380000993011F490E105C09A3011F090E001C0B8
:1038100096E18091140C981729F09093140C03C032
:103820001092140C90E0892F0895EF92FF920F935D
:103830001F93CF93DF93F894E090B802F090B90211
:1038400078948701A895F894C091B802D091B902F4
:103850007894CE01801B910B409718F00E94CD1BED
:103860008E010E94DC1B882331F4CE19DF09C05180
:10387000D74240F389E1CDB7DEB7E6E00C9453625E
:103880000F931F93CF93DF939C01EB018A0101C03B
:10389000A895F999FDCFCE01B9014FE150E00E9402
:1038A0002F631F8E8881992787FD90950E94626201
:1038B000892B21F4CE01B8010E949262DF91CF9151
:1038C0001F910F9108950F931F93CF93DF939C0146
:1038D000EB018A0101C0A895F999FDCFCE01B9018C
:1038E0004FE050E00E942F631F868881992787FD53
:1038F00090950E946262892B21F4CE01B8010E944A
:103900009262DF91CF911F910F910895EF92FF92F4
:103910000F931F93142F052FF62EE72E01C0A895A5
:10392000F999FDCF0E943F639B01AC012F3F8FEFC0
:1039300038078FEF48078FEF580741F4212F302FBA
:103940004F2D5E2DC901DA019C01AD01B901CA01FB
:103950001F910F91FF90EF9008951F93CF93DF93E6
:10396000EC010E949962182F813414F580910103B3
:1039700090910203019711F4A895FECF81E090E0A9
:1039800090930203809301038FEB92E0BE010E94AB
:1039900092628091BF028093C60011501093000381
:1039A00081E08093FF028091C10080668093C10016
:1039B000DF91CF911F9108951F93BC01FC010190ED
:1039C0000020E9F731971E2F181B11340CF5809158
:1039D000010390910203019711F4A895FECF81E0B5
:1039E00090E090930203809301038FEB92E00E949A
:1039F0000B638091BF028093C600115010930003A7
:103A000081E08093FF028091C10080668093C100B5
:103A10001F9108951F93482F792F162F613444F575
:103A20008091010390910203019711F4A895FECFB4
:103A300081E090E090930203809301032FEB32E04A
:103A4000E62FFF27E7FDF095C901642FAF010E9423
:103A5000CA628091BF028093C60011501093000388
:103A600081E08093FF028091C10080668093C10055
:103A70001F9108950000000008952D9A2F980000CE
:103A800000002F9A90E087FF02C02D9A01C02D9868
:103A90002F98000000002F9A9F5F983011F0880F38
:103AA000F2CF08951F93CF93DF93182FEB018091EE
:103AB0008C04813021F4CB010E94D83EEC01F894B3
:103AC0002F9A5F9A80E30E943D1D5F982F9A5F9A1C
:103AD0001F73812F80640E943D1D80E0D7FF02C0CC
:103AE0002D9A01C02D982F98000000002F9A0000F9
:103AF00000008F5F803119F0CC0FDD1FEFCF5F9892
:103B00002D985F9A000000001E9BFECF5F985F9883
:103B10007894DF91CF911F9108951F93CF93DF93F6
:103B2000C0E0D1E012E0688179812296812F0E9465
:103B3000521D1F5F1530B9F7DF91CF911F91089586
:103B4000FF920F931F93182F062FF72EBA010E9492
:103B5000521D812F8F5F602F7F2D0E94521D1F915C
:103B60000F91FF900895F8942F9A5F9A8F73806851
:103B70000E943D1D80E020E030E02F980000000012
:103B80002F9A00000000220F331F1E9921608F5FC3
:103B9000803199F7932F5F98789480918C048130CD
:103BA00021F4822F0E94D83E9C01C90108951F93E1
:103BB000CF93DF9380E00E94B31D8050904419F4AE
:103BC00081E080938C0482E00E94B31D8F5F9F4F41
:103BD00061F012E0C0E0D1E0812F0E94B31D888324
:103BE000998322961F5F1530B9F7DF91CF911F910E
:103BF00008959F92AF92BF92CF92DF92EF92FF9281
:103C00000F931F93182F042FB52EA62E972E0E94C8
:103C1000B31D6C01812F8F5F0E94B31D7C018FEF5C
:103C2000C8168FEFD8068FEFE8068FEFF80641F43D
:103C3000202F3B2D4A2D592DC901DA016C017D0140
:103C4000B601C7011F910F91FF90EF90DF90CF90C9
:103C5000BF90AF909F9008951F1D1F1E1F1E1F1F16
:103C60001E1F1E1FCF93DF93EC012C964AE834D021
:103C70006627772736E4AEE6B1E0532F537009F09C
:103C80001197321729F078F56A0F7B1F3395F3CF20
:103C90004CE022D0E8E5FCE330E0C89531963130C5
:103CA00011F451110A94321720F4600D711D3395EF
:103CB000F4CF402D439510D02150A8F0620F711D14
:103CC0008827992748E108D015D04CE305D012D0B9
:103CD0002CE302D00FD00BC03A912A912417310562
:103CE00040F00F900F906FEF7FEF8FEF9FEFDF911E
:103CF000CF91089551E2AA1B08F4A40FA7959795B8
:103D00008795779567955A95B9F7620F711D811D53
:103D1000911D0895CF93DF93FC0120813181428171
:103D20005381CC27DD2757FD3CC0C5E1DCE06CE3C7
:103D30003CD00882198239D00A821B8268E135D0D2
:103D40000C821D82F9012C5F3F4F67E02ED00C865C
:103D50001D869F01A6E4EEE6F1E0BA2FB37009F0EC
:103D600031972E173F0720F02E1B3F0BA395F3CF63
:103D7000AA871B862E873F87E8E5FCE3AA27C8951C
:103D80003196A13011F4B1110A942015310520F0BB
:103D900020193109A395F3CFA887198623952E837F
:103DA0003F83CE01DF91CF910895002470E2220F6E
:103DB000331F441F551F001C061610F0061A2395CA
:103DC0007A95A9F70895EAECF4E08281813041F414
:103DD00080819181019791838083892B09F41282DC
:103DE0003D9685E0E233F80781F70895CF92DF92A0
:103DF000EF92FF920F931F936B017C018AE290E098
:103E0000909399048093980480E00E94171582E0B3
:103E10006DEC7FE10E94F1148FEF66E070E00E948C
:103E2000011600E011E0C80166E070E00E94E915AB
:103E300086E098E00E94BF1581E090E00E94BF15E7
:103E400080E098E00E94BF1586E00E94B21584E0F1
:103E50000E94B21581E090E00E94BF15C80166E0A3
:103E600070E00E94E9156091290570912A05809102
:103E70002B0590912C050E94D01580E066E070E043
:103E80000E940116C701B6010E94D0158CEC9FE17B
:103E90000E94EF161F910F91FF90EF90DF90CF904F
:103EA0000895EF92FF920F931F93CF93DF937B01BF
:103EB0008C01E901E0ECF4E020E080819181A281B5
:103EC000B3818E159F05A007B10711F4922F0DC085
:103ED0002F5F3D96283089F7CD2BF9F0909128057A
:103EE000892F8F5F8770809328058DE0989FF00160
:103EF0001124E054FB4FEF012496DA0186E00D9087
:103F000009928150E1F7E082F1820283138380EB12
:103F100094E09387828781E08487CDB7DEB7E6E0BF
:103F20000C945362ACE1B0E0E8E9FFE10C9431623B
:103F3000CE0101966CE170E00E949B158F819885FF
:103F40000E94D83E4C016F85788989899A890E94A0
:103F5000DC3E5B016C01698D7A8D8B8D9C8D0E949E
:103F6000DC3E7B018C0189819A810E94D83E0197B9
:103F700009F071C08B819C810E94D83E805098408E
:103F800009F069C08091290590912A05A0912B051F
:103F9000B0912C05E816F9060A071B0709F05BC06B
:103FA000CE01439660E071E046E050E00E9412636B
:103FB000009709F050C0AE14BF04C006D10611F43A
:103FC00082E04AC08E01075F1F4FC601B501A801FC
:103FD00021E030E00E94511F81E088169104D9F55C
:103FE0008CE190E090939904809398048EE090E0A7
:103FF0000E94841681E090E00E94BF1580E098E066
:104000000E94BF1586E00E94B21584E00E94B2159E
:1040100082E090E00E94BF1580E091E066E070E0F1
:104020000E94E9156091290570912A0580912B0560
:1040300090912C050E94D015C80166E070E00E94A6
:10404000E915CE010F9664E070E00E94E91586E064
:1040500098E00E949A2080E06C96ECE00C944D620F
:10406000EF92FF920F931F93E090A004F090A104B1
:104070000091A2041091A30420912D0530912E05EA
:1040800040912F0550913005DA01C9018E299F29F1
:10409000A02BB12B8F5F9F4FAF4FBF4F49F48AE9E1
:1040A00094E06FEF70E046E050E00E94E56235C0BA
:1040B0008091290590912A05A0912B05B0912C059E
:1040C0008E259F25A027B12782239323A423B523E0
:1040D0000097A105B10511F421E009C0E090310578
:1040E000F0903205009133051091340522E0E0ECA8
:1040F000F4E08485813099F480819181A281B3813B
:104100008E159F05A007B10751F4AAE9B4E03496D3
:1041100086E001900D928150E1F720E005C03D96C8
:1041200085E0E832F80729F7822F1F910F91FF9061
:10413000EF9008950F931F938C01809198049091B4
:1041400099040E96909399048093980480E090E0EF
:104150000E9484168AE994E066E070E00E94E91506
:1041600080E091E066E070E00E94E915C8010E94DD
:10417000BF1588ED99E10E94EF161F910F910895E8
:10418000AEE0B0E0E6ECF0E20C943A62CE010196CB
:104190000E949B198823F1F0AAE9B4E0FE0137964A
:1041A00086E001900D928150E1F78D859E850E94F9
:1041B000D83E28E08030920711F411E00CC0865000
:1041C000984031F40E94921F182F0E949E1603C03F
:1041D0000E949E1610E0812F2E96E3E00C9456620A
:1041E000A8E0B0E0E6EFF0E20C94396282E290E001
:1041F0000E945F16CE01019668E070E00E949B1558
:104200008981809338058A8180933905609198046B
:104210007091990482E290E00E94E317892B81F06B
:104220008AE390E00E945F160E947F1560933A0532
:1042300070933B0580933C0590933D0587E057C004
:1042400080913805883031F16D817E818F8198852C
:104250000E94DC3E9B01AC0160933A0570933B05E4
:1042600080933C0590933D0580913805833019F487
:104270000E94EB183BC08530C9F58091390581302B
:10428000A9F52093310530933205409333055093BF
:1042900034052CC0409198045091990482E290E03A
:1042A00062E270E00E940D1882E290E00E948416A3
:1042B00080E00E94B21580E00E94B21580E090E09C
:1042C0000E94BF15609198047091990482E290E079
:1042D0000E94F2178C0184E290E00E948416C801CB
:1042E0000E94BF1581E00E94D52101C08AE0289676
:1042F000E4E00C945562A0E0B0E0E1E8F1E20C9457
:104300003462B82EEB016A01E4EBF4E0EE24FF2402
:104310008701308121813296C901A0E0B0E0E80E2A
:10432000F91E0A1F1B1F84E0E03CF80791F781E0AB
:10433000B81651F480E00E941715C752D64E80E09F
:10434000BE010E94F11403C0CE010E945F16C60197
:104350000E948D179C0140E050E02E0D3F1D401F34
:10436000511F203080E0380781E0480780E058077F
:10437000A0F0CA0140E050E0A0E0B0E0280F391FF3
:104380004A1F5B1F203080E0380781E0480780E04B
:10439000580718F0C90101969C0120953095C90174
:1043A000CDB7DEB7E9E00C945062ACE1B0E0EBEDE4
:1043B000F1E20C943962182F80919804909199043D
:1043C000449690939904809398048EE090E00E9424
:1043D000841680E095E40E94BF1580919804909126
:1043E00099040E94BF1580913505909136050E9471
:1043F000BF1580E090E40E94BF1580E40E94B215D2
:10440000812F0E94B21580E090E00E94BF1560915C
:10441000290570912A0580912B0590912C050E9409
:10442000D0156091A0047091A1048091A204909194
:10443000A3040E94D0158EE090E064E170E00E9439
:10444000F2178C0188E190E00E948416C8010E9456
:10445000BF150E943020882309F443C0DE01119665
:10446000E8E9F4E09CE101900D929150E1F782308F
:1044700049F4609131057091320580913305909136
:10448000340508C06091A0047091A1048091A20439
:104490009091A3040E94F61E0E949E160E944B1B40
:1044A0008C01A8950E94C020882311F00E949E16BE
:1044B0000E943020882311F420E008C00E944B1B8A
:1044C000801B910B8858934160F326E0A8E9B4E083
:1044D000FE0131968CE101900D928150E1F722238B
:1044E00029F480E098E00E949A2020E08091350530
:1044F0009091360501969093360580933505822F6D
:104500006C96E4E00C945562A4E1B0E0EAE8F2E2D3
:104510000C9437620E94C020882309F4A1C0823025
:1045200011F485E09DC08EE090E064E170E00E94AF
:10453000E317892B09F091C08EE090E00E945F168E
:10454000CE01019664E170E00E949B1569897A8929
:104550008B899C890E94DC3E7B018C0120912D057A
:1045600030912E0540912F05509130058981682F9B
:1045700070E0CB01807F90708034910509F06DC0B0
:104580008091290590912A05A0912B05B0912C05C9
:10459000E816F9060A071B0799F02E293F29402B38
:1045A000512B2F5F3F4F4F4F5F4F51F08FEFE8166A
:1045B0008FEFF8068FEF08078FEF180709F04DC04F
:1045C0006F707070660F771F660F771F60933705E7
:1045D0008B819C810E94D83E20913705821B9109D6
:1045E00090939904809398046D857E858F85988932
:1045F0000E94DC3E6093A0047093A1048093A20407
:104600009093A304E092A404F092A5040093A6045E
:104610001093A70480913705853120F0845190E0F4
:104620000E94A3186091A0047091A1048091A2043B
:104630009091A3044AE954E020E030E00E94511F29
:104640008A85813011F482E00BC0813111F483E05E
:1046500007C0863011F484E003C00E949E1680E0FB
:104660006496E6E00C945362A0E0B0E0EAE3F3E283
:104670000C943662D82EEB017A0184E190E0E80ECA
:10468000F91EF0929904E09298048CEE9FEFE80EE8
:10469000F91E82E290E00E9484168D819E810E9424
:1046A000BF158F8198850E94BF1569857A858B8596
:1046B0009C850E94D0156D857E858F8598890E9486
:1046C000D01580E50E94B2158D2D8F730E94B21512
:1046D00084EB95E00E94BF1560E070E080E090E020
:1046E0000E94D0156091290570912A0580912B05B3
:1046F00090912C050E94DC3E6093B4047093B50445
:104700008093B6049093B70469817A818B819C81F0
:104710000E94DC3E6093B8047093B9048093BA049D
:104720009093BB041092BC0486E08093BD048091FA
:104730009804909199040E94D83E9093BF0480936E
:10474000BE04409198045091990481E062E270E0C7
:104750000E947B218C0182E390E00E948416C801B4
:104760000E94BF1586E00E94D521682F882301F59D
:104770008D2D90E083709070892B41F089859A850A
:10478000AB85BC850196A11DB11D0EC0E114F104DD
:1047900079F0970140E050E089859A85AB85BC852A
:1047A000820F931FA41FB51F89879A87AB87BC8789
:1047B000862FCDB7DEB7E7E00C945262A2E1B0E0FD
:1047C000E4EEF3E20C943B622091A8043091A9043A
:1047D000C901A0E0B0E08A839B83AC83BD83809154
:1047E000AA049091AB049F838E83398728871A8609
:1047F0001B861C861D868091B0049091B104A09107
:10480000B204B091B3040196A11DB11D8E879F879C
:10481000A88BB98B84E0BE016F5F7F4F40E050E012
:104820000E9434236296E2E00C945762A8E0B0E064
:10483000ECE1F4E20C9431627C018091AC04909143
:10484000AD040E945F1600E010E06E010894C11CE8
:10485000D11C2AE6A22E27E0B22EAE0CBF1C92E09D
:10486000892E9924939453C0C60165E070E04AE014
:104870000E948818080F191FC60167EE70E00E9499
:104880008962892B91F4E114F10419F086E696E02F
:1048900002C086E695E06BEF70E04AE00E9488185F
:1048A000080F191FF501908232C0C60162EE70E058
:1048B00044E050E00E94A262892B19F4F501808245
:1048C00026C089818D30E1F48A818A30C9F48091D3
:1048D000AE049091AF0408171907C8F0EE0CFF1C46
:1048E00086E697E0E80EF91E81E090E0F7019183FB
:1048F000808315C00F5F1F4F0E9460158A3039F00A
:104900008091AE049091AF040817190798F3809135
:10491000AE049091AF040817190708F4A5CF2896A4
:10492000ECE00C944D62CF93DF93EC01009719F00B
:1049300026E636E002C026E635E0FE01EE0FFF1F58
:10494000DF0143E0AA0FBB1F4A95E1F7AE0FBF1F7F
:10495000A25CBA4F1C9211961D921D921D921C9240
:10496000149716961C921E92159718961C921E92DA
:1049700017971D961D921D921D921C92509780E0D4
:1049800091E0D901AC011D9241505040E1F7EA5944
:10499000F84F11821082C659D84F1882DF91CF91FB
:1049A0000895A6E2B0E0E7EDF4E20C942D620091E8
:1049B000370510E0025F1F4FCE01439664E170E0BF
:1049C0000E949B158B899C890E94D83E9093A904D4
:1049D0008093A8048D899E890E94D83E9093AB0451
:1049E0008093AA046F89788D898D9A8D0E94DC3E10
:1049F0006093B0047093B1048093B2049093B304B5
:104A00002F8D2695269530E0C801820F931F909335
:104A1000AD048093AC048091980490919904821B1A
:104A2000930B9093AF048093AE046091A0047091B7
:104A3000A1048091A2049091A3040E94DC3E6093A3
:104A4000B4047093B5048093B6049093B704609156
:104A5000A4047091A5048091A6049091A7040E94DB
:104A6000DC3E6093B8047093B9048093BA049093C9
:104A7000BB041092BC0486E08093BD04809198042E
:104A8000909199040E94D83E9093BF048093BE04F5
:104A9000409198045091990480E0B8010E947B21D4
:104AA000892B09F099C198A1992309F495C16090C7
:104AB000A0047090A1048090A2049090A304E090C0
:104AC000A804F090A904A090AA04B090AB040EE34F
:104AD00015E0CC24DD246FEF7FEF2E010894411CFC
:104AE000511CD201F80182E101900D928150E1F751
:104AF000AE81BF81E885F9852A813B814C815D814A
:104B00008981882331F48FEF6F3F780711F4B60164
:104B10000BC0261537054805590531F4EE15FF057C
:104B200019F4AA15BB05C1F00894C11CD11C0E5E76
:104B30001F4FE2E0CE16D104A1F6FFEF6F3F7F07D3
:104B400041F06B01C094D0948CE9C8168FEFD80661
:104B500019F40E94DE23FFC0D7FE47C091FF3FC17A
:104B60008091620590916305A816B90609F037C1D6
:104B7000C094D094C601880F991F8C0143E0000FA8
:104B8000111F4A95E1F7080F191F025C1A4FF8012F
:104B90006182728283829482B682A582F086E782E5
:104BA00081E080830E94673EF80161877287838776
:104BB00094878091B0049091B104A091B204B09117
:104BC000B3040196A11DB11D85879687A787B08B79
:104BD0008CE3818B82E1B80140E050E00E943423F5
:104BE000F82E882309F4FCC053C091FF03C00E9433
:104BF000DE234DC092FF0FC0B601660F771FCB01B9
:104C000023E0880F991F2A95E1F7680F791F625CEE
:104C10007A4F84E038C090FF3FC0C601880F991FCB
:104C20008C01B3E0000F111FBA95E1F7080F191FAF
:104C3000025C1A4FF80120818091B0049091B10478
:104C4000A091B204B091B3040196A11DB11D858756
:104C50009687A787B08B223079F480E1B80140E0D5
:104C600050E00E94342381E1B80140E050E00E940E
:104C70003423F82E85E0A1C0233019F0263009F046
:104C8000AEC080E1B80140E050E00E943423F82E2D
:104C9000C6010E949324A4C093FF5FC08091AE041C
:104CA0009091AF04009711F480E055C05601AA0C12
:104CB000BB1C8501F3E0000F111FFA95E1F70A0D07
:104CC0001B1D025C1A4FF8012081213019F482E08B
:104CD000808302C0223011F0FF243CC0A0E0B0E08D
:104CE0002091B0043091B1044091B2045091B304CA
:104CF000820F931FA41FB51FF80185879687A7878A
:104D0000B08B2581368180916205909163052817CB
:104D10003907B1F480E1B80140E050E00E9434234B
:104D2000F82EC6010E941624F501EA59F84F808139
:104D30009181019779F4C6010E940445F82E0AC0BA
:104D400081E1B80140E050E00E943423F82E83E076
:104D5000F80180838F2DF82E43C094FF40C0C60118
:104D6000880F991F8C0173E0000F111F7A95E1F7EE
:104D7000080F191F025C1A4FF8018081813011F46D
:104D800082E022C08230E1F48091AE049091AF04C1
:104D9000892B59F080E1B80140E050E00E943423B3
:104DA000F82EC6010E9416241BC081E1B80140E024
:104DB00050E00E943423F82E83E0F801808310C075
:104DC000833021F486E0F801808309C0853039F40E
:104DD000C6010E94932403C068E0F62E01C0FF24A0
:104DE0008F2DA696E0E10C944962CF93DF9308964D
:104DF000909399048093980482E290E00E94841634
:104E00008091AA049091AB040E94BF158091A804E0
:104E10009091A9040E94BF158091980490919904E3
:104E20000E94BF1580E090E00E94BF1560912905A7
:104E300070912A0580912B0590912C050E94DC3EF3
:104E40006093B4047093B5048093B6049093B70450
:104E50006091A0047091A1048091A2049091A30498
:104E60000E94DC3E6093B8047093B9048093BA0446
:104E70009093BB041092BC0481E18093BD048091A7
:104E80009804909199040E94D83E9093BF04809317
:104E9000BE04409198045091990481E062E270E070
:104EA0000E947B21EC01009711F4CFEFDFEF88E245
:104EB00090E00E948416CE010E94BF1581E10E94FD
:104EC000D521DF91CF910895A0E1B0E0EAE6F7E2C5
:104ED0000C943762CE01099668E070E00E949B1541
:104EE00089859A850E94D83E9093A9048093A8044E
:104EF0008B859C850E94D83E9093AB048093AA0436
:104F00008D859E850E94D83E8C01085010401093DC
:104F1000AF040093AE04085F1F4F80913705E82E61
:104F2000FF248EE090E0E80EF91E8F859889892B8A
:104F3000B9F16091A0047091A1048091A2049091B4
:104F4000A3040E94DC3E6093B4047093B504809384
:104F5000B6049093B7046091A4047091A504809165
:104F6000A6049091A7040E94DC3E6093B80470935D
:104F7000B9048093BA049093BB041092BC0481E1FD
:104F80008093BD048D859E859093BF048093BE045D
:104F900080E0B701A8010E947B21892B09F04AC05B
:104FA000C70108969093AD048093AC042091AA04A5
:104FB0003091AB042B37310519F40E9450343DC0B9
:104FC0002532310519F40E94273C37C044E02030D7
:104FD000340719F40E94C32D30C02434310519F46C
:104FE0000E94832B2AC02938310519F40E940B2F07
:104FF00024C02151374201F50E945F168E010F5FD8
:105000001F4FC80167E070E00E949B15C80166EF62
:1050100070E047E050E00E94A262892B69F48AE2C6
:1050200090E00E9484168DEE90E00E94B6180E94D7
:10503000F526FFCF89E001C080E06096E6E00C94A1
:1050400053628091290890912A08A0912B08B09171
:105050002C088093A0049093A104A093A204B09381
:10506000A30483E490E09093A9048093A80484E4CB
:1050700090E09093AB048093AA048AE290E00E94AF
:10508000841660E076E081E091E00E94D0150E94F5
:10509000673E60933D0870933E0880933F0890936D
:1050A00040080E94D01580E090E00E94BF1580E08B
:1050B00090E00E94BF1560E070E080E090E00E9408
:1050C000D01580E06CE070E00E94011680E091E075
:1050D00066E070E00E94E91580E06AEC70E00E94F2
:1050E000011663E673E582E893E60E94D01581E03D
:1050F00095E30E94BF1584E00E94B21582E30E94EE
:10510000B21584E00E94B2156091290570912A05BC
:1051100080912B0590912C050E94D01586E30E946A
:10512000B21584E00E94B2156091290870912A0896
:1051300080912B0890912C080E94D0158FEF0E942F
:10514000B21580E06CE270E00E9401168CE291E002
:105150000E94F52608950F931F9381E080935408D1
:105160008FEF9FEFAFEFBFEF8093A0049093A10468
:10517000A093A204B093A30483E490E09093A904C5
:105180008093A80484E490E09093AB048093AA04F5
:1051900010922D0510922E0510922F0510923005B9
:1051A0001092290510922A0510922B0510922C05B9
:1051B0001092DD091092DE091092DF091092E009C9
:1051C0001092310510923205109233051092340579
:1051D000109225081092260810922708109228088D
:1051E000109221081092220810922308109224088D
:1051F00010922D0810922E0810922F08109230084D
:105200001092290810922A0810922B0810922C084C
:105210001092390810923A0810923B0810923C08FC
:10522000109231081092320810923308109234080C
:1052300010923508109236081092370810923808EC
:105240001092490810924A0810924B0810924C088C
:10525000109257080E94673E60933D0870933E0885
:1052600080933F08909340088AE290E00E94841661
:1052700060E076E081E091E00E94D01560913D0809
:1052800070913E0880913F08909140080E94D0158F
:1052900060E070E880E090E00E94D01580E060E17E
:1052A00070E00E94011600E011E0C80166E070E0C5
:1052B0000E94E91580E06AEC70E00E94011663E646
:1052C00073E582E893E60E94D01581E095E30E94A1
:1052D000BF1581E00E94B2158DE30E94B21587E0F0
:1052E0000E94B21581E00E94B215C80166E070E02C
:1052F0000E94E9158FEF0E94B21580E06FE270E026
:105300000E9401168CE291E00E94F5261F910F91F8
:1053100008950F931F93182F80935408883129F014
:105320008FEF9FEFAFEFBFEF08C0809129089091FA
:105330002A08A0912B08B0912C088093A004909388
:10534000A104A093A204B093A304133051F00E94CF
:10535000673E60933D0870933E0880933F089093AA
:105360004008EDECF9E001900020E9F73197ED5CA1
:10537000F9400E2F0F5F83E490E09093A90480938F
:10538000A80484E490E09093AB048093AA048AE29A
:1053900090E00E94841660E076E081E091E00E9457
:1053A000D01560913D0870913E0880913F08909122
:1053B00040080E94D01580E090E00E94BF1518318F
:1053C00019F080E090E802C080E090E00E94BF15F4
:1053D0006091290570912A0580912B0590912C05EB
:1053E0000E94D01580E06CE070E00E94011680E021
:1053F00091E066E070E00E94E91580E06AEC70E000
:105400000E94011663E673E582E893E60E94D015D8
:1054100081E095E30E94BF1583E00E94B2158CE005
:105420000E94B215802F0E94B2158DEC99E0602F7A
:1054300070E00E94E915133019F582E30E94B2155D
:1054400084E00E94B2158091AC049091AD04409626
:105450000E945F160E947F150E94D01586E30E946D
:10546000B21584E00E94B2156091290870912A0853
:1054700080912B0890912C080E94D01519E115C03D
:10548000163111F015E211C082E30E94B21584E0DA
:105490000E94B21560911D0870911E0880911F082E
:1054A000909120080E94D0151FE187E30E94B21559
:1054B00086E00E94B21581E00E94B21583E00E944E
:1054C000B21586E00E94B21583E30E94B2158AE30A
:1054D0000E94B2158BE30E94B2158DE30E94B215B3
:1054E00087E00E94B21581E00E94B21580E091E051
:1054F00066E070E00E94E9158FEF0E94B215101B64
:1055000080E0612F70E00E9401168CE291E00E9421
:10551000F5261F910F910895EF92FF920F931F931D
:105520008091550890915608892B59F4A8E0B1E074
:10553000EDE1F1E082E101900D928150E1F760E050
:10554000DCC080915408813031F0863121F08831FF
:1055500011F08931D9F5E0905108F090520800E03F
:1055600010E088E091E06DE171E00E94753FE61A7D
:10557000F70A080B190BE0924D08F0924E080093C1
:105580004F08109350081E141F0410061106F4F063
:1055900080915408813049F0863159F48091570840
:1055A0008F5F80935708833018F00E94AB2803C0A8
:1055B00086E10E948929682FA8E0B1E0EDE1F1E0E1
:1055C00082E101900D928150E1F701C060E0E0902E
:1055D0004908F0904A0800914B0810914C08D801F6
:1055E000C7010196A11DB11D0297A105B10508F4DF
:1055F00084C08091410890914208A0914308B091E5
:105600004408209145083091460840914708509140
:1056100048080097A105B10591F10197A109B109C9
:105620008093410890934208A0934308B0934408A4
:105630002150304040405040209345083093460868
:1056400040934708509348080894E108F10801097D
:105650001109E0924908F0924A0800934B08109310
:105660004C080097A105B10509F047C088E10E94E8
:105670008929682F882309F040C06CE03EC0089457
:10568000E108F1080109110921153105410551050C
:1056900009F1DA01C9010197A109B109809345080F
:1056A00090934608A0934708B0934808E0924908B1
:1056B000F0924A0800934B0810934C080097A105FC
:1056C000B105D9F489E10E948929682F8823A9F4BA
:1056D0006DE013C0E0924908F0924A0800934B082D
:1056E00010934C08E114F1040105110531F40E94F6
:1056F000AB28682F882309F46EE0862F1F910F9145
:10570000FF90EF900895ACE1B0E0E9E8FBE20C9483
:10571000376280915408882309F4E8C1873109F47D
:10572000E5C18091AC049091AD0480519F4F0E94DF
:105730005F160E946015182F8F3F09F4C5C00E94A4
:105740006015082F153341F4813009F0D6C10E944D
:10575000601580935308EDCF113071F4843009F057
:10576000CCC10E947F15609321087093220880931A
:10577000230890932408DDCF133071F4843008F4AB
:10578000BCC10E947F156093250870932608809302
:105790002708909328081FC0163371F4843008F44A
:1057A000ACC10E947F156093290870932A088093EA
:1057B0002B0890932C080FC01630A1F4843008F405
:1057C0009CC10E947F1560932D0870932E088093D2
:1057D0002F0890933008043009F4ABCF802F90E06D
:1057E00004976FC0133309F04BC0843009F0A1CF88
:1057F0000E947F157B018C016093390870933A08F1
:1058000080933B0890933C0880913508909136082E
:10581000A0913708B09138080097A105B105B1F4FF
:10582000C801B7012BE633E040E050E00E94AF61D1
:1058300028EE33E040E050E00E94EE61209335080E
:1058400030933608409337085093380880913108D8
:1058500090913208A0913308B09134080097A105C7
:10586000B10509F066CF16950795F794E794E09295
:105870003108F0923208009333081093340859CF5E
:105880001A3371F4843009F054CF0E947F1560936D
:10589000310870933208809333089093340849CFCD
:1058A0001B3371F4843009F044CF0E947F1560935C
:1058B000350870933608809337089093380839CFAD
:1058C00090E00E94A31835CF8091AC049091AD0474
:1058D00004960E945F16809154089091530881307D
:1058E000B9F4923009F004C10E947F1520913D085F
:1058F00030913E0840913F0850914008621773076D
:105900008407950709F0F4C083E00E948929F1C05B
:10591000953009F0D9C00E947F1520913D08309143
:105920003E0840913F085091400862177307840772
:10593000950709F0DDC087E1809354088091AC049D
:105940009091AD0440960E945F160E947F15AB01B6
:10595000BC014093290550932A0560932B05709351
:105960002C0588E090E00E946D6380912108909161
:105970002208A0912308B091240880932D059093CC
:105980002E05A0932F05B0933005809125089091A6
:105990002608A0912708B09128088093310590939C
:1059A0003205A0933305B093340580912D08909172
:1059B0002E08A0912F08B09130088093DD099093B4
:1059C000DE09A093DF09B093E0098091310890913E
:1059D0003208A0913308B091340880934108909325
:1059E0004208A0934308B0934408809135089091F1
:1059F0003608A0913708B0913808809345089093F5
:105A00004608A0934708B0934808809139089091C0
:105A10003A08A0913B08B0913C08809349089093C4
:105A20004A08A0934B08B0934C088F5F9F4FAF4F2D
:105A3000BF4F21F41092560810925508DE011196BE
:105A4000E8E9F4E08CE101900D928150E1F760917A
:105A5000290570912A0580912B0590912C050E94B3
:105A6000F61E0E949E160E944B1B8C01A8950E9458
:105A7000C020813019F40E949E1609C0823039F48A
:105A80000E9421288823B1F40E94AB2813C00E94F1
:105A90004B1B801B910B8D54914040F38091E10989
:105AA0008150823030F481E090E09093E609809359
:105AB000E50980E0A8E9B4E0FE0131969CE101909F
:105AC0000D929150E1F715C0963091F40E947F1528
:105AD00020913D0830913E0840913F085091400888
:105AE000621773078407950719F407C080E001C0A7
:105AF0008FE06C96E6E00C9453620E94AB28F9CFDD
:105B0000AF92BF92DF92EF92FF920F931F93DF93BA
:105B1000CF930F92CDB7DEB7F82EE92E9C01590135
:105B20008EE2D82E0E946015982F882331F40894B5
:105B3000A108B108F501108219C0807C803C11F0E9
:105B400085010AC00E94601511C099830E946015EA
:105B5000F80181938F019981802F8A198917A8F301
:105B6000A90EB11CF501D1925F01DCCF8F2D9E2DC6
:105B70000F90CF91DF911F910F91FF90EF90DF90E9
:105B8000BF90AF900895ACE4B0E0E9ECFDE20C9476
:105B90002D628091AC049091AD040E945F16CE01FD
:105BA00001966CE070E00E949B1589819A810E94A9
:105BB000D83E2091C2093091C3098217930709F09A
:105BC0006AC08D819E810E94D83E6C01EE24FF2424
:105BD0003DE2A32EB12CAC0EBD1E2DE0822E912CE9
:105BE0008C0E9D1E14C0C5010E94802D0E946D1553
:105BF0008C010E946D150130110531F4019721F4DB
:105C0000C401B5010E940B630894E11CF11CEC1463
:105C1000FD0448F38F8198850E94D83E3C01EE2414
:105C2000FF249DE2492E512C4C0E5D1E31C0C20155
:105C30000E94802D0E946D158C010E946D154C01F3
:105C40000E947F155B016C010E946D1501301105EA
:105C5000D1F421E082169104B1F48430910599F4D5
:105C60000E947F15AB01BC014093C4095093C50944
:105C70006093C6097093C709CE010D969601850100
:105C80000E94E93108C00E94A3180894E11CF11C8D
:105C9000E614F70460F280E0C45BDF4FE0E10C94AF
:105CA0004962AF92BF92DF92EF92FF920F931F93E0
:105CB000CF93DF93182F092F8091DD099091DE0992
:105CC000A091DF09B091E0098093A0049093A10412
:105CD000A093A204B093A30485E390E09093A90459
:105CE0008093A80480E094E09093AB048093AA048E
:105CF0000E94673E7093C3096093C2098AE290E0F4
:105D00000E9484168091C2099091C3090E94BF1518
:105D100080E091E00E94BF1581E090E00E94BF15F5
:105D200080E090E00E94BF1580E090E00E94BF15E7
:105D300080E090E00E94BF15212F302FC901EC01B7
:105D400040E1A42EB12C7E010E2D0C1BF701D0805A
:105D5000FEE2DF1631F0DD2021F00894E11CF11C99
:105D6000F3CF802F0E94B21510E0CE01B8010E943F
:105D7000E9150F5F1F4FA00EB11EDD2019F0E701DE
:105D80002196E1CF80E00E94B21581E090E00E9470
:105D9000BF1581E090E00E94BF15C50101960E94E9
:105DA000F526DF91CF911F910F91FF90EF90DF903B
:105DB000BF90AF9008951F930E946015182F115443
:105DC0001295107F0E94601581548F70812B1F9156
:105DD00008950F931F93CF93DF93EC0100E0899117
:105DE00090E00E947662182F85958595859585951A
:105DF0008F5B0E94B2151F70812F8F5B0E94B215BE
:105E00000F5F003161F780E00E94B215DF91CF9102
:105E10001F910F910895ACE1B0E0E1E1FFE20C9435
:105E20002D628091AC049091AD040E945F16CE016A
:105E300001966CE070E00E949B158B819C810E9412
:105E4000D83E9C018F709070892B11F082E1EEC0DA
:105E500037FF5AC089819A810E94D83E2091C20999
:105E60003091C3098217930709F0DFC08F819885AD
:105E70000E94D83E019711F080E1D8C00E946015C1
:105E8000803211F081E1D2C08E01035F1F4FC80143
:105E9000902E892E2DE1E22EF12CEC0EFD1E0E949B
:105EA000DB2EF80181938F01EE15FF05C1F71C8EE3
:105EB0000E9460150E946D158C010E946D157C0179
:105EC0000E947F155B016C010032110509F0ADC025
:105ED000F1E0EF16F10409F0A8C00E946D150E94D0
:105EE0006D150E947F15AB01BC014093C40950930E
:105EF000C5096093C6097093C709892D982D96012D
:105F000085010E94E93191C020703877232B09F078
:105F10008CC08091AE049091AF04C29709F085C007
:105F200089819A810E94D83E4C018D819E810E9478
:105F3000D83E5C01CC24DD249DE0692E712C6C0ED2
:105F40007D1E8DE1482E512C4C0E5D1E31C00E94ED
:105F50006015803209F069C083010E94DB2EF801D0
:105F600081938F01E415F505C1F71C8E0E94601521
:105F70000E946D157C010E946D150197B1F4F0E24D
:105F8000EF16F10451F4C3016DEC79E00E94026355
:105F9000009759F400E015E84FC081E2E816F104DB
:105FA00021F48D858A3209F445C00894C11CD11CA6
:105FB000CA14DB0460F239C086E090E00E94BF158D
:105FC00080E090E00E94BF156091290570912A053C
:105FD00080912B0590912C050E94D0158EE390E0C6
:105FE00021C08DE390E00E94BF1581E00E94B215B0
:105FF0008DEC99E06FE070E00E94E91580E00E946E
:10600000B21580E094E00E94BF1580E091E066E068
:1060100070E00E94E91580E064E270E00E940116E1
:1060200085E790E00E94F52601C080E06C96E0E1F3
:106030000C94496200E014E88AE290E00E94841621
:10604000C4010E94BF15C8010E94BF1580E090E006
:106050000E94BF1581E090E00E94BF1580E090E0B3
:106060000E94BF1580E090E00E94BF1580E20E9470
:10607000B215CE010D960E94E92EC7010E94BF15F0
:1060800081E090E00E94BF1568E572E080E090E05A
:106090000E94D015E0E2EE16F10409F0A2CF8CCFF9
:1060A0000F931F938C0180912D0590912E05A09147
:1060B0002F05B091300580959095A095B0952091D1
:1060C000290530912A0540912B0550912C05822BF2
:1060D000932BA42BB52B8093A0049093A104A093A1
:1060E000A204B093A30489E890E09093A90480935C
:1060F000A8049093AB048093AA040E94673E709317
:10610000C3096093C2098AE290E00E9484168091DC
:10611000C2099091C3090E94BF1580E191E00E94DD
:10612000BF1581E090E00E94BF1580E090E00E94E2
:10613000BF1580E090E00E94BF1580E090E00E94D3
:10614000BF1580E20E94B215C8010E94E92E80E2CC
:1061500090E00E94BF1581E090E00E94BF1582E3AD
:1061600090E00E94F5261F910F910895ECE9F8E068
:1061700084818130A1F480819181A281B3810097D3
:10618000A105B10561F00197A109B109808391834F
:10619000A283B3830097A105B10509F41482B996CF
:1061A00089E0E43EF80721F70895A9E2B0E0EBEDBD
:1061B000F0E30C9435627C0108E718E06E01089466
:1061C000C11CD11CD601F80189E201900D928150C9
:1061D000E1F789A5813059F4C601B7010E94026335
:1061E000009729F429A13AA14BA15CA10AC0075D3F
:1061F0001F4F89E0003C180729F720E030E040E01D
:1062000050E0B901CA01A996E8E00C945162CF931D
:10621000DF938091CA09813001F5C8E5D8E0CE014D
:1062200064EC79E00E94E23E813009F4C3C0FE01D3
:1062300001900020E9F73197EC1BFD0B709738F4C3
:10624000CE016EE270E00E94F762009711F084E0E8
:1062500001C082E08093CA09A9C0823009F588E5AF
:1062600098E00E94D5306093C4097093C50980936B
:10627000C6099093C709611571058105910509F05B
:1062800099C00E944B1B9093C1098093C00988E577
:1062900098E00E945030282F1092C90983E053C023
:1062A000833079F58091C4099091C509A091C60900
:1062B000B091C7090097A105B10509F07BC00E9404
:1062C0004B1B2091C0093091C109821B930B885E42
:1062D000934008F46BC08091C9098F5F8093C9090E
:1062E000833020F02091F0072D5E61C00E944B1B8F
:1062F0009093C1098093C00988E598E00E945030CE
:1063000053C0843019F588E598E00E94D530609339
:10631000C4097093C5098093C6099093C709611594
:1063200071058105910509F045C00E944B1B9093B2
:10633000C1098093C00988E598E00E94512E282F5A
:106340001092C90985E08093CA0931C0853071F582
:106350008091C4099091C509A091C609B091C7095F
:106360000097A105B10531F50E944B1B2091C00992
:106370003091C109821B930B885E9340B8F08091E5
:10638000C9098F5F8093C909833020F02091F007FD
:10639000295E0DC00E944B1B9093C1098093C009D8
:1063A00088E598E00E94512E282F01C020E080E06F
:1063B00090E003C020E081E090E09093CC098093CE
:1063C000CB09019711F41092CA09822FDF91CF9166
:1063D0000895A0E0B0E0EFEEF1E30C942F62EC0141
:1063E0006A017B014801590100E010E089E2682E52
:1063F000712C069DC001079D900D169D900D1124D6
:106400008858974FBE010E940263009739F10F5FD1
:106410001F4F0830110569F72091C809822F8F5F3F
:1064200087708093C80930E089E290E0289F80015E
:10643000299F100D389F100D11240858174FC801BF
:10644000BE010E940B63F801C0A2D1A2E2A2F3A296
:1064500084A295A2A6A2B7A281E080A7CDB7DEB79D
:10646000EEE00C944B62A8E0B0E0E9E3F2E30C94B8
:1064700033626D837E838F83988719821A821B8291
:106480001C8229813A814B815C81F8EEAF2EE3E0DA
:10649000BE2ECC24DD24EE24FF2400E010E00E9478
:1064A0003A5B952FB901842F2896EAE00C944F624D
:1064B000A4E2B0E0EEE5F2E30C9435621091F0074F
:1064C0001093F10700E0B5E0EB2EF12CEC0EFD1E71
:1064D0006E010894C11CD11C1F5F1370E12FF0E006
:1064E000EE0FFF1FEE59FE4F65917491C7010E9498
:1064F0000B63C701B6010E94E23E813041F48981FD
:106500009A81AB81BC810097A105B10519F0109368
:10651000F00703C00F5F0430F9F6A496E8E00C948E
:106520005162AF92BF92CF92DF92EF92FF920F93A0
:106530001F936093A0047093A1048093A20490938E
:10654000A3048BE790E09093A9048093A804909310
:10655000AB048093AA048AE290E00E94841683E24E
:106560000E94B21580E067E270E00E940116F89484
:10657000E090000CF090010C0091020C1091030CC3
:106580006091FE0B7091FF0B882777FD8095982F07
:106590000E9433325B016C0178946093020870931F
:1065A0000308809304089093050880E89EE7AAEA10
:1065B000B3E8E80EF91E0A1F1B1FC801B7010E94AD
:1065C000D015C601B5010E94D01580E390E00E946D
:1065D000F5261F910F91FF90EF90DF90CF90BF9025
:1065E000AF9008951F931091F309112309F480C00F
:1065F0001130A1F48091F007E82FF0E0EE0FFF1FBB
:10660000EE59FE4F6591749188E598E00E940B6306
:106610001093CA0982E08093F3096AC0123089F5A9
:106620008091CB099091CC09019709F061C010923B
:10663000CC091092CB096091C4097091C509809171
:10664000C6099091C70960936C0770936D0780939A
:106650006E0790936F0710921A080E949132182FBC
:10666000882351F483E08093F3090E944B1B90939D
:1066700013088093120802C01092F3090E94583246
:1066800038C01330A9F50E944B1B2091120830919D
:106690001308821B930B2091140830911508821760
:1066A000930730F180911A088F5F80931A08833026
:1066B00040F010937C011091F107145E0E94A80B2A
:1066C00018C060916C0770916D0780916E07909172
:1066D0006F070E949132182F882339F40E944B1BB8
:1066E000909313088093120804C01092F30901C01C
:1066F00010E0812F1F9108958091E409823019F4F0
:1067000082E091E004C0833041F48EEF90E00E947B
:10671000B61880E00E94B215089560912905709125
:106720002A0580912B0590912C050E94D015089583
:10673000AF92BF92CF92DF92EF92FF920F931F938F
:106740008091F6079091F707A091F807B091F907AB
:106750008093A0049093A104A093A204B093A304F7
:106760008BE790E09093A9048093A8049093AB04E6
:106770008093AA048091F4099091F509892B19F46A
:1067800005EE10E102C005E211E08AE290E00E940D
:106790008416802F0E94B215812F0E94B21560913D
:1067A00016087091170820E030E84FE0C9018623F1
:1067B0009723892B29F4415019F036952795F6CF68
:1067C000842F0E94B21586EF0E94B2156091FA07DD
:1067D0007091FB078091FC079091FD070E94D015F6
:1067E0006091FE077091FF07809100089091010869
:1067F0000E94D0150E947C3360911008709111089E
:1068000080E090E00E9433327B018C0160910A08A5
:1068100070910B0880910C0890910D086058714898
:1068200085459C470E94D015C801B7010E94D0152C
:1068300080E060E170E00E940116F894E090000CA6
:10684000F090010C0091020C1091030C6091FE0B72
:106850007091FF0B882777FD8095982F0E94333227
:106860005B016C01789480E89EE7AAEAB3E8E80E41
:10687000F91E0A1F1B1FC801B7010E94D015C601CF
:10688000B5010E94D01580E390E00E94F5261F918B
:106890000F91FF90EF90DF90CF90BF90AF90089551
:1068A000A7E6B0E0E6E5F4E30C942B628091AC043B
:1068B0009091AD040E945F16CE01819660E370E076
:1068C0000E949B1599A1892F8770843009F034C4E8
:1068D0008091F309882309F4B4C7892F807C8093C1
:1068E00006019AA1803C21F0992311F0903158F0D3
:1068F00082E080937C011092CA091092F3090E94F1
:10690000A80B8BE19FC79F5F909307016DA17EA1AC
:106910008FA198A50E94DC3E6093FA077093FB0755
:106920008093FC079093FD0769A57AA58BA59CA58C
:106930000E94DC3E6093FE077093FF07809300087F
:1069400090930108FE01E05CFF4F90812FAD5EAD9A
:106950006DAD7CADABADDAAC99ACFE01EC5BFF4F3D
:10696000C080FE01ED5BFF4FB080FE01EE5BFF4F8C
:10697000A080FE01EF5BFF4F7080FE01E85BFF4FE0
:106980008081FE01E95BFF4F3081FE01EA5BFF4F32
:106990004081FE01EB5BFF4FE081E82EE91A91E0B8
:1069A0008E1508F090E0832F821B21E0381708F045
:1069B00020E0F82EF91A91E08F1508F090E0292BCD
:1069C000842F851B31E0481708F030E0082F021BA8
:1069D00091E0801708F090E0392B8E2F861B21E084
:1069E000E81708F020E0182F131B91E0811708F03A
:1069F00090E0292B8C2D871B31E0C81608F030E081
:106A0000B82FB21B91E08B1708F090E0392B8B2D3B
:106A10008A1B21E0B81608F020E0A82FA31B91E004
:106A20008A1708F090E0292B8A2D8D1991E0A8167D
:106A300008F090E0F82FF21B21E08F1708F020E01B
:106A4000922BE72DE919E91B9701A8016B2F7A2FEB
:106A50008F2F9E2F52F52E2D2F5F81E02E1508F0DF
:106A600080E0382F3F0D81E03F1508F080E0482F8F
:106A7000400F81E0401708F080E0582F510F81E06F
:106A8000511708F080E0682F6B0F81E06B1708F05A
:106A900080E0782F7A0F81E07A1708F080E08F0F7E
:106AA00091E08F1708F090E09E0F01E00E94B55A28
:106AB000622E532E442E352E262E62967FAF62977D
:106AC00063968FAF639764969FAF6497FE01E45B14
:106AD000FF4FC080FE01E55BFF4FB080FE01E65B2B
:106AE000FF4FA080FE01E75BFF4F7080FE01E05B7F
:106AF000FF4F0081FE01E15BFF4FF080FE01E25B92
:106B0000FF4F9080FE01E35BFF4F8080809106087D
:106B100090910708A0910808B09109088058914801
:106B2000A545BC47182F8D8B9E8BAF8BB88F60917E
:106B30000E0870910F0880E090E00E943332698B5C
:106B40007A8B8B8B9C8B872F3B89492F5E897F8922
:106B5000E88DD02ED61A91E00D1508F090E02F2D7B
:106B6000281B822F21E0F81608F020E0E82EE91A11
:106B700091E08E1508F090E0292B892D831B31E0E0
:106B8000981608F030E0F82EF21A91E08F1508F010
:106B900090E0392B882D841B21E0881608F020E036
:106BA000082F031B91E0801708F090E0292B3C2D63
:106BB000311B132F91E0C31608F090E0B12FB21BE8
:106BC00081E01B1708F080E0982B8B2D851B21E0BE
:106BD000B81608F020E0A82FA91B91E08A1708F04A
:106BE00090E0292B8A2D871B91E0A81608F090E0F1
:106BF000F82FF21B21E08F1708F020E0922B7E1A6D
:106C0000E72DE91B2D2D3E2D4F2D502F6B2F7A2F69
:106C10008F2F9E2F52F52D2D2F5F81E02D1508F01F
:106C200080E0382F3E0D81E03E1508F080E0482FCF
:106C30004F0D81E04F1508F080E0582F500F81E094
:106C4000501708F080E0682F6B0F81E06B1708F099
:106C500080E0782F7A0F81E07A1708F080E08F0FBC
:106C600091E08F1708F090E09E0F01E00E94B55A66
:106C7000A32FB42F152F062FF72ED82EC22EC60CF9
:106C8000F1E0C21608F0F0E03A2F350DE1E03A17D6
:106C900008F0E0E0EF2EE30E21E0E31608F020E03C
:106CA000E22B4B2F440D31E04B1708F030E0AE2FB4
:106CB000A40F21E0A41708F020E0322B512F530D30
:106CC00041E0511708F040E0F32FF50F21E0F517F0
:106CD00008F020E0422B602F620D31E0601708F0D1
:106CE00030E0E42FE60F21E0E61708F020E0322B39
:106CF00062967FAD62977F0D41E07F1508F040E01E
:106D0000532F570F21E0571708F020E0422B6396CE
:106D10008FAD63978D0D21E08D1508F020E0480FB1
:106D200031E0481708F030E0232B64968FAD64976C
:106D3000980F290FC98AEA8AAB8BFC8BED8B5E8B8F
:106D40004F8B288F4D885E886F88788C89899A89C7
:106D5000AB89BC894C015D01CC24DD2476019C010A
:106D6000A50160E070E080E090E002E00E94365A09
:106D7000122F232E65964FAF659766965FAF669785
:106D800067966FAF679768967FAF689769968FAF82
:106D900069976A969FAF6A9705E00E94365AA32FBB
:106DA000B42F052F6B966FAF6B976C967FAF6C9778
:106DB0006D968FAF6D976E969FAF6E97322E311A8C
:106DC000F1E0231508F0F0E03A2F3219E1E0A317C3
:106DD00008F0E0E0132F1F1B21E0311708F020E03E
:106DE000E22B4B2F65969FAD6597491B31E0B41799
:106DF00008F030E0B42FBE1B21E04B1708F020E074
:106E0000322B502F6696AFAD66975A1B41E005179F
:106E100008F040E0052F031B21E0501708F020E0A8
:106E2000422B6B966FAD6B976796EFAD67976E1BB6
:106E300031E06B96FFAD6B97F61708F030E0962FB8
:106E4000941B21E0691708F020E0322B6C967FAD8F
:106E50006C9768962FAD6897721B41E06C968FAD6A
:106E60006C97871708F040E0A72FA31B21E07A1743
:106E700008F020E0422B6D968FAD6D976996EFADCF
:106E800069978E1B21E06D96FFAD6D97F81708F09E
:106E900020E0E82FE41B31E08E1708F030E0232BD0
:106EA0006E96FFAD6E976A963FAD6A97F31BF21B25
:106EB000232C280C31E0231408F030E0812F890DB9
:106EC00041E0811708F040E0380F51E0381708F032
:106ED00050E0452B8B2F8A0D51E08B1708F050E0C6
:106EE000480F61E0481708F060E0562B202F2B0D6B
:106EF00081E0201708F080E0520F61E0521708F09F
:106F000060E0682B690F71E0691708F070E07A0F94
:106F100081E07A1708F080E08E0F91E08E1708F07C
:106F200090E0222D9F0F03E00E94365A298F3A8F5E
:106F30004B8F5C8F6D8F7E8F8F8F98A3ED8CFE8C27
:106F40000F8D18A180911B0190911C01892BC9F410
:106F500080911B0890911C08009799F0A301920161
:106F600077FE07C022273327A901241935094609CE
:106F70005709A0E0B0E082179307A407B5070CF407
:106F800060C48701F8948091000C9091010CA0914D
:106F9000020CB091030C840D951DA61DB71D8093A6
:106FA000000C9093010CA093020CB093030C809101
:106FB000FE0B9091FF0B8E0D9F1D9093FF0B809306
:106FC000FE0B8091FE0B9091FF0B97FF2AC08091E2
:106FD000000C9091010CA091020CB091030C1816BA
:106FE00019061A061B06ECF48091000C9091010C16
:106FF000A091020CB091030C0197A109B1098093F3
:10700000000C9093010CA093020CB093030C8091A0
:10701000FE0B9091FF0B88519C4F9093FF0B809338
:10702000FE0B8091000C9091010CA091020CB0918C
:10703000030C80930A0890930B08A0930C08B0935C
:107040000D088091FE0B9091FF0B90931108809397
:1070500010088091000C9091010CA091020CB0914D
:10706000030C0196A11DB11D80930D0C90930E0C85
:10707000A0930F0CB093100C10927D0181E08093CF
:10708000130C789477FE0AC0101611063CF408948D
:10709000411C511C611C711C085E1340D301C201CC
:1070A00080509048AF4FBF4F80509040A140B040BB
:1070B00038F08FEF9FE79093F3078093F20704C0B7
:1070C0005092F3074092F2071093F5070093F407EC
:1070D0008091FC09882361F1C301B20128EE33E0FD
:1070E00040E050E00E94AF619B01AC01C801AA27BB
:1070F00097FDA095BA2F820F931FA41FB51FB7FD50
:1071000004C0B801620F731F0AC0C301B20128E1B5
:107110003CEF4FEF5FEF0E94AF61601B710B70930C
:10712000FB096093FA096D54714014F081E001C0CD
:1071300082E08093FC097FC3833009F0D6C0292FF9
:1071400028738091F4099091F509019701F5509009
:107150000601522A40900701E0900A08F0900B08BF
:1071600000910C0810910D0880E89EE7AAEAB3E8A8
:10717000E80EF91E0A1F1B1F60911008709111087C
:1071800080E090E00E9433323B014C010BC040ECA8
:10719000542E522A662477244301EE24FF248701CB
:1071A00030E1432EA0900608B0900708C090080870
:1071B000D090090820900E0830900F088AE290E0E5
:1071C0000E948416852D84600E94B215842D0E9431
:1071D000B2158BA10E94B21586EF0E94B21560E035
:1071E00070E080E090E00E94D01560E070E080E008
:1071F00090E00E94D0150E947C33C801B7010E9424
:10720000D015C401B3010E94D0158091F40990916A
:10721000F509019799F4CE0181968C01085D1F4F05
:1072200020E3E22EF12CE80EF91ED8018D918D019C
:107230000E94B2150E151F05C1F70CC060E070E08A
:1072400080E090E00E94D01560E070E080E090E087
:107250000E94D01580E89EE7AAEAB3E8A80EB91EFE
:10726000CA1EDB1EC601B5010E94D015B10180E027
:1072700090E00E9433320E94D0158091F4099091E1
:10728000F509019739F0AA24BB246501EE24FF24F7
:1072900087011EC0F894E090000CF090010C009162
:1072A000020C1091030C80E89EE7AAEAB3E8E80E0E
:1072B000F91E0A1F1B1F6091FE0B7091FF0B8827A0
:1072C00077FD8095982F0E9433325B016C01789492
:1072D000C801B7010E94D015C601B5010E94D015A2
:1072E00080E390E00E94F526ADC2853009F0A9C286
:1072F0008091E409813009F0A4C2892F807C8093B9
:1073000006019AA1803C09F49CC2992309F499C210
:10731000903109F496C29F5F909307016DA17EA101
:107320008FA198A50E94DC3E6093FA077093FB073B
:107330008093FC079093FD0769A57AA58BA59CA572
:107340000E94DC3E6093FE077093FF078093000865
:1073500090930108FE01E05BFF4FD080FE01E15BEE
:10736000FF4FC080FE01E25BFF4FA080FE01E35BA8
:10737000FF4F10813D2DD9822C2DCA829A2DAB82D0
:10738000812F1C83FE01E45BFF4FD080FE01E55B93
:10739000FF4FC080FE01E65BFF4FA080FE01E75B70
:1073A000FF4F1081DD82CE82AF821887032FF22E2D
:1073B000E92EB82E832F822B892B8B298D298C299E
:1073C0008A29812B09F43DC2F8948091000C909198
:1073D000010CA091020CB091030C80589148A54576
:1073E000BC478D839E83AF83B8876091FE0B7091FD
:1073F000FF0B882777FD8095982F0E943332698391
:107400007A838B839C83789489812A813B814C8108
:107410005D81AE81BF819884F02FF81B91E00F173A
:1074200008F090E08F2D821B21E0F81608F020E094
:10743000E82FE91B91E08E1708F090E0292B8E2DA4
:10744000831B31E0E81608F030E0782F721B91E0E2
:10745000871708F090E0392B8B2D841B21E0B8169C
:1074600008F020E0682F631B91E0861708F090E099
:10747000292B8D2D851B31E0D81608F030E0582FD0
:10748000521B91E0851708F090E0392B8C2D8A1B58
:1074900021E0C81608F020E0482F431B91E0841734
:1074A00008F090E0292B8A2D8B1B91E0A81608F09C
:1074B00090E0382F321B21E0831708F020E0922B58
:1074C0001919191BF983EA837B836C835D834E83CF
:1074D0003F8318874D805E806F80788489819A8190
:1074E000AB81BC814C015D01CC24DD2476019C0183
:1074F000A50160E070E080E090E002E00E94365A72
:10750000122F232E6F964FAF6F97A0965FAFA09765
:10751000A1966FAFA197A2967FAFA297A3968FAFC8
:10752000A397A4969FAFA49705E00E94365AA32F75
:10753000B42F052FA5966FAFA597A6967FAFA697F8
:10754000A7968FAFA797A8969FAFA897322E311A0C
:10755000F1E0231508F0F0E03A2F3219E1E0A3172B
:1075600008F0E0E0132F1F1B21E0311708F020E0A6
:10757000E22B4B2F6F969FAD6F97491B31E0B417ED
:1075800008F030E0B42FBE1B21E04B1708F020E0DC
:10759000322B502FA096AFADA0975A1B41E0051794
:1075A00008F040E0052F031B21E0501708F020E011
:1075B000422BA5966FADA597A196EFADA1976E1B37
:1075C00031E0A596FFADA597F61708F030E0962FAD
:1075D000941B21E0691708F020E0322BA6967FADBE
:1075E000A697A2962FADA297721B41E0A6968FADEB
:1075F000A697871708F040E0A72FA31B21E07A1772
:1076000008F020E0422BA7968FADA797A396EFAD89
:10761000A3978E1B21E0A796FFADA797F81708F058
:1076200020E0E82FE41B31E08E1708F030E0232B38
:10763000A896FFADA897A4963FADA497F31BF21BA5
:10764000232C280C31E0231408F030E0812F890D21
:1076500041E0811708F040E0380F51E0381708F09A
:1076600050E0452B8B2F8A0D51E08B1708F050E02E
:10767000480F61E0481708F060E0562B202F2B0DD3
:1076800081E0201708F080E0520F61E0521708F007
:1076900060E0682B690F71E0691708F070E07A0FFD
:1076A00081E07A1708F080E08E0F91E08E1708F0E5
:1076B00090E0222D9F0F03E00E94365A29873A87D7
:1076C0004B875C876D877E878F87988BED84FE84E0
:1076D0000F85188980911B0190911C01892BC9F499
:1076E00080911B0890911C08009799F0A3019201CA
:1076F00077FE07C022273327A90124193509460937
:107700005709A0E0B0E082179307A407B5070CF46F
:1077100098C09701F8948091000C9091010CA09171
:10772000020CB091030C840D951DA61DB71D80930E
:10773000000C9093010CA093020CB093030C809169
:10774000FE0B9091FF0B8E0D9F1D9093FF0B80936E
:10775000FE0B8091FE0B9091FF0B97FF2AC080914A
:10776000000C9091010CA091020CB091030C181622
:1077700019061A061B06ECF48091000C9091010C7E
:10778000A091020CB091030C0197A109B10980935B
:10779000000C9093010CA093020CB093030C809109
:1077A000FE0B9091FF0B88519C4F9093FF0B8093A1
:1077B000FE0B8091000C9091010CA091020CB091F5
:1077C000030C80930A0890930B08A0930C08B093C5
:1077D0000D088091FE0B9091FF0B90931108809300
:1077E0001008789477FE0AC0121613063CF4089429
:1077F000411C511C611C711C285E3340D301C20125
:1078000080509048AF4FBF4F80509040A140B04053
:1078100038F08FEF9FE79093F3078093F20704C04F
:107820005092F3074092F2073093F5072093F40744
:1078300081E08093130C81E090E09093080C80939A
:10784000070C80E0C959DF4FE2E10C944762809158
:10785000F4099091F509892B11F480E008958AE2EA
:1078600090E00E948416F8946091000C7091010CD5
:107870008091020C9091030C789460587148854572
:107880009C470E94D01584E090E00E94F526089560
:10789000DB01982F92959F702AE631E0F901E90FFC
:1078A000F11DE491EC938F70280F311DF901849143
:1078B00011968C93119712961C921297CB010895F2
:1078C000DB01292F22952F704AE651E0FA01E20FE1
:1078D000F11DE491EC939F70FA01E90FF11DE49121
:1078E0001196EC931197982F92959F70FA01E90FDA
:1078F000F11DE4911296EC9312978F70480F511D71
:10790000FA01849113968C93139714961C921497F2
:10791000CB010895DA01292F22952F704AE651E014
:10792000FA01E20FF11DE491EC939F70FA01E90F67
:10793000F11DE4911196EC931197982F92959F70F9
:10794000FA01E90FF11DE4911296EC9312978F70F2
:10795000FA01E80FF11DE4911396EC931397872F2A
:1079600082958F70FA01E80FF11DE4911496EC9363
:1079700014977F70FA01E70FF11DE4911596EC93CF
:107980001597862F82958F70FA01E80FF11DE4910B
:107990001696EC9316976F70460F511DFA0184915D
:1079A00017968C93179718961C921897CD010895E7
:1079B000282FDB0164E60E94CE61392F822F0E94BE
:1079C000CE61805DFD018193832F6AE00E94CE61CC
:1079D000805D11968C931197832F0E94CE61905DEC
:1079E00091831282CD010895A0E0B0E0EAEFFCE3BC
:1079F0000C943662482FF92EE62ED72E862F972F1D
:107A00009C01E901E0E1F7E200E010E0842F9F2D06
:107A1000BF010E94DA61262F842F9F2DBF010E9493
:107A2000DA61482FF92E205D2993CF016AE070E0DA
:107A30000E94DA61FB010F5F1F4F0430110531F71F
:107A4000405D488319828E2D9D2DCDB7DEB7E7E0CE
:107A50000C945262A0E0B0E0E0E3FDE30C942E62EF
:107A6000062F772E4C01642E552E842F952F9C01C6
:107A7000E901C12C8AECD82E8AE9E82E8BE3F82E96
:107A8000AA24BB24602F772DC401A70196010E9470
:107A9000EE61122F602F772DC401A70196010E947D
:107AA000EE61062F772E4C01105D1993C701B601C8
:107AB0002AE030E040E050E00E94EE61C901DA01C6
:107AC0006C017D010894A11CB11C89E0A816B104C9
:107AD000C9F6005D08831982862D952DCDB7DEB7D6
:107AE000EFE00C944A62EF92FF920F931F938B0189
:107AF0009C01F42EE52E97FD04C0842F952FFC01E8
:107B00000CC030952095109501951F4F2F4F3F4F7A
:107B1000842F952FFC018DE28193C901B801AF013B
:107B20000E942A3D8F2D9E2D1F910F91FF90EF9067
:107B300008951F93CF93DF93EC0120E030E040E005
:107B400050E01881812F80538A30C8F4CA01B901EE
:107B50002AE030E040E050E00E94AF619B01AC01C0
:107B6000812F992787FD9095C097AA2797FDA0950B
:107B7000BA2F280F391F4A1F5B1F2196E2CF2030F2
:107B800080E0380781E0480780E0580720F02FEFB9
:107B90003FEF40E050E0C901DF91CF911F91089580
:107BA000982F8154863010F487E307C0892F8156BF
:107BB000863010F487E501C080E3981B892F089573
:107BC000FF920F931F938C01FC0180810E94D03D96
:107BD000F82EF29490EFF922F80181810E94D03DB5
:107BE0008F708F291F910F91FF900895EF92FF9250
:107BF0000F931F938C01FC0180810E94D03DF82ED1
:107C0000F29430EFF322F80181810E94D03D8F7011
:107C1000F82AF80182810E94D03DE82EE29420EFFC
:107C2000E222F80183810E94D03D8F708E299F2D22
:107C30001F910F91FF90EF900895CF92DF92EF92F6
:107C4000FF920F931F938C01FC0180810E94D03D15
:107C5000C82EC29470EFC722F80181810E94D03DE6
:107C60008F70C82AF80182810E94D03DD82ED2940C
:107C700060EFD622F80183810E94D03D8F70D82A10
:107C8000F80184810E94D03DF82EF29450EFF52245
:107C9000F80185810E94D03D8F70F82AF801868115
:107CA0000E94D03DE82EE29440EFE422F801878163
:107CB0000E94D03D8F708E29682F7F2D8D2D9C2D99
:107CC0001F910F91FF90EF90DF90CF900895EF926A
:107CD000FF920F931F9380917E0190917F01A0915D
:107CE0008001B09181017C018D012BE0EE0CFF1C25
:107CF000001F111F2A95D1F7E826F9260A271B270E
:107D00008091820190918301A0918401B0918501BD
:107D100080937E0190937F01A0938001B0938101B5
:107D20008091860190918701A0918801B09189018D
:107D30008093820190938301A0938401B093850185
:107D400080918A0190918B01A0918C01B0918D015D
:107D50008093860190938701A0938801B093890155
:107D60009C01AD01F3E15695479537952795FA9516
:107D7000D1F7282739274A275B272E253F2540277B
:107D80005127EF2CF02E012F11272E253F254027BC
:107D9000512720938A0130938B0140938C0150939B
:107DA0008D01B901CA011F910F91FF90EF900895C5
:107DB000282F892F922F0895362F272F692F782F5C
:107DC000C9010895A0E2B0E0E8EEFEE30C94316250
:107DD0009C015B018E010F5F1F4FC801B9010E941A
:107DE0000B63CC24DD247601980140E1842E912C94
:107DF0008C0E9D1EF80180818E3291F41082C90193
:107E00000E94993DA0E0B0E08C299D29AE29BF29B0
:107E1000CC24D82EE92EFA2E98012F5F3F4F2BC08D
:107E20008823E9F4CE0101960817190731F4F5010A
:107E3000108211821282138210C0F8011082C901CF
:107E40000E94993DA0E0B0E08C299D29AE29BF2970
:107E5000F50180839183A283B38381E013C09927C6
:107E600087FD9095C0970A9730F0F5011082118236
:107E70001282138206C00815190519F00F5F1F4FF3
:107E8000B9CF80E0A096ECE00C944D62CF92DF92E7
:107E9000EF92FF920F931F936B01E82E8A01892FB7
:107EA000BA010E94D83C5EE2F52EF801F382B801D7
:107EB0006C5F7F4F8E2D0E94D83CF801F782B8018D
:107EC000685F7F4F8D2D0E94D83CF801F386B80182
:107ED000645F7F4F8C2D0E94D83CC8011F910F9189
:107EE000FF90EF90DF90CF900895CF92DF92EF92C6
:107EF000FF920F931F936B010E94321E7B018C0136
:107F0000C6010E94321E9B01AC012E193F09400B95
:107F1000510BB901CA011F910F91FF90EF90DF90B3
:107F2000CF900895A4E0B0E0E8E9FFE30C94396253
:107F3000162F072F0E94321E209177013091780171
:107F40004091790150917A01260F371F481F591F20
:107F500029833A834B835C83CE0101960E948A1E5B
:107F6000AC01009711F480E00BC0812F902F9C0191
:107F7000D901FA0182E101900D928150E1F781E08F
:107F80002496E4E00C945562A4E0B0E0EAECFFE350
:107F90000C943562D62EC72E79018A010E94321EBA
:107FA0006E197F09800B910B69837A838B839C8385
:107FB000CE0101960E948A1EAC01009711F480E068
:107FC0000BC08D2D9C2D9C01D901FA0182E10190FD
:107FD0000D928150E1F781E02496E8E00C94516223
:107FE000EF92FF920F931F93E82EF62E8A01FA94D8
:107FF0000E94151CF8018083813131F48E2D8F5F32
:10800000F81660F480E00AC0823111F08E2D06C0AF
:10801000EE2011F48F2D02C08E2D81501F910F91F3
:10802000FF90EF900895A0E0B0E0E9E1F0E40C9457
:108030002C62C82E362E7A01B22EE8010E94B31AA5
:10804000EB2DFF27E7FDF095EE0DFF1D1082F701E8
:108050009081892F80538A3010F4182F08C0892FFF
:108060008154863010F010E002C0192F1753A895E4
:108070001B9BFDCF81E00E94661A219711F08AE0D8
:1080800001C080E1012F112707FD1095DC2CC0E015
:10809000D0E04B2C552447FC5094882E992487FC23
:1080A000909434010894610871085701AC0EBD1E0C
:1080B0008D2D632D0E947A1A0A30110518F4802F35
:1080C000805D02C0802F895C0E944A1A0E945E1A5D
:1080D0000E94151C813141F40F5F1F4F08151905CF
:1080E0004CF000E010E006C0823179F401501040FD
:1080F00017FD83010A30110518F4802F805D02C03E
:10810000802F895CF5018083D0CF833151F5219692
:10811000D394F701EC0FFD1F8081992787FD90957F
:108120000E946262892B11F42196D394C415D5055F
:108130001CF0DC2CC0E0D0E0F701EC0FFD1FE0816B
:108140008E2F80538A3040F08E2F8154863010F06D
:1081500080E002C08E2F8753082F112707FD10954E
:10816000A4CF843119F401E010E005C0893109F091
:108170009CCF00E010E080E00E94661AC801CDB7F5
:10818000DEB7E1E10C9448621F920F920FB60F9296
:1081900011248F939F9382E083BD1092B20081E0FF
:1081A0008CBB1DBA8AE08093120C88EC8093060C7D
:1081B00084E690E090931108809310089093FF0B51
:1081C0008093FE0B9F918F910F900FBE0F901F9089
:1081D00018951F920F920FB60F9211240F900FBE99
:1081E0000F901F9018951F920F920FB60F921124A7
:1081F0000F900FBE0F901F9018951F920F920FB601
:108200000F9211242F933F938F939F93AF93BF931C
:1082100080917D018823F9F080917D0181508093C8
:108220007D0180917D018823B1F480910D0C9091A6
:108230000E0CA0910F0CB091100C0196A11DB11D58
:1082400080930D0C90930E0CA0930F0CB093100C18
:1082500081E08093130C8091FE0B9091FF0B0196AF
:108260009093FF0B8093FE0B8091FE0B9091FF0B80
:10827000885E9340DCF11092FF0B1092FE0B809110
:10828000130C882359F180910D0C90910E0CA09144
:108290000F0CB091100C80930A0890930B08A093D8
:1082A0000C08B0930D088093000C9093010CA093E0
:1082B000020CB093030C21E030E03093050C2093C6
:1082C000040C88EC80937D018091130C823021F4A2
:1082D0003093080C2093070C1092130C8091E40942
:1082E000882321F01092110810921008BF91AF91CD
:1082F0009F918F913F912F910F900FBE0F901F90E4
:1083000018951F920F920FB60F9211248F939F937F
:108310008091B8029091B90201969093B90280932E
:10832000B8028091060C882359F08091060C815088
:108330008093060C8091060C882311F481E08DBB9C
:108340009F918F910F900FBE0F901F9018951F92C5
:108350000F920FB60F9211248F939F93EF93FF9379
:108360008091C0009091C6008C7179F480910404D2
:10837000E82FF0E0ED5FFC4F90838F5F8093040463
:10838000809105048F5F80930504FF91EF919F9189
:108390008F910F900FBE0F901F9018951F920F9204
:1083A0000FB60F9211242F938F939F93EF93FF9308
:1083B000209100032223B9F09091FF02E92FF0E011
:1083C000E154FD4F80818093C6009F5F9093FF0230
:1083D000822F815080930003882329F48091C1006B
:1083E0008F7D8093C100FF91EF919F918F912F918D
:1083F0000F900FBE0F901F9018951F920F920FB6FF
:108400000F9211248F9380910003882349F4809167
:10841000C1008F7B8093C100109202031092010370
:108420008F910F900FBE0F901F901895CF93DF93F1
:10843000EC0163E27BE044E050E00E94A262892B01
:1084400011F481E017C0CE016FE17BE043E050E022
:108450000E94A262892B11F482E00CC0CE0168E177
:108460007BE046E050E00E94A262892B11F483E099
:1084700001C080E0DF91CF910895CF93DF93019702
:1084800019F0C0E0D0E005C083E49DE00E94B6187A
:10849000EC0187E29DE00E94B6189E01280F391F6B
:1084A000C901DF91CF910895A0E0B0E0EAE5F2E4E0
:1084B0000C942D623B01E82FFF27E7FDF095EE0FAE
:1084C000FF1FEF52F84F4590549086EE9DE00E94BA
:1084D000B6184C01C2010E94B618EC0188EC9DE070
:1084E0000E94B6185C01C2010E94B6186C018AEAAB
:1084F0009DE00E94B6187C01C2010E94B6188C0152
:1085000086E99DE00E94B618C80DD91DCA0DDB1D75
:10851000CC0DDD1DCE0DDF1DC00FD11FC80FD91F23
:1085200081E068167104A9F486E89DE00E94B618FF
:108530007C01C2010E94B6188C018BE69DE00E946E
:10854000B6189701200F311F2C0F3D1F280F391F20
:1085500007C086E69DE00E94B6189C012C0F3D1FC7
:10856000C901CDB7DEB7E0E10C944962EF92FF920A
:108570000F931F93182F86E390E00E9484168CEED1
:1085800091E00E94B6187C01E12FFF27E7FDF095EE
:10859000EE0FFF1FE55BF74F859194910E94B6188F
:1085A0008C018CEF9DE00E94B6180E0D1F1D080F68
:1085B000191FC8011F910F91FF90EF900895A0E03F
:1085C000B0E0E5EEF2E40C943362082F86E390E02D
:1085D0000E9484168CEE91E00E94B6185C01C02FB8
:1085E000DD27C7FDD095CC0FDD1FFE01E55BF74F02
:1085F000859194910E94B6188C0188E39EE00E94B8
:10860000B6186C01FE01EF52F84F859194910E94CB
:10861000B6187C018AE29EE00E94B6180A0D1B1D66
:108620000C0D1D1D0E0D1F1D080F191FC801CDB704
:10863000DEB7EAE00C944F62AF92BF92CF92DF9226
:10864000EF92FF920F931F938C01F62EE72E89EC89
:108650009CE00E94B6185C01C8010E94B6188C010B
:108660008FEB9CE00E94B6186C01EF2DFE2DDF0110
:108670000D900020E9F71197AE1BBF0B8F2D9E2D9B
:10868000BD010E94E9157C0184EB9CE00E94B618B4
:108690000A0D1B1D0C0D1D1D0E0D1F1D080F191F92
:1086A000C8011F910F91FF90EF90DF90CF90BF9086
:1086B000AF900895A4E0B0E0E0E6F3E40C943B62F0
:1086C000BE016F5F7F4F0E94D83CCE01029662E0F0
:1086D00070E00E94E9152496E2E00C945762A8E04D
:1086E000B0E0E5E7F3E40C942F627C01FC018081AB
:1086F0009181BE016F5F7F4F0E94F43CCE010296D4
:1087000064E070E00E94E9153C018FE20E94B2151E
:10871000F70182810E945A438C018FE20E94B215B8
:10872000F70183810E945A434C0180E20E94B215F6
:10873000F70184810E945A435C018AE30E94B215CA
:10874000F70185810E945A436C018AE30E94B215A9
:10875000F70186810E945A43080D191D0B5F1F4FB8
:108760000A0D1B1D0C0D1D1D080F191F060D171DD1
:10877000C8012896EEE00C944B62A8E0B0E0E3EC70
:10878000F3E40C942B626C0180E29DE00E94B61829
:108790009E838D83F601808191810E94B6188C01A1
:1087A00082E09DE00E94B61898878F83F60182814F
:1087B00093810E94B6181C0189EF9CE00E94B618B4
:1087C0002C01F60184817E010894E11CF11CB701A3
:1087D0000E94D83CF70101900020E9F73197EE198B
:1087E000FF09BF010E94E9153C018BEE9CE00E944D
:1087F000B6184C01F6018581B7010E94D83CF701FB
:1088000001900020E9F73197EE19FF09BF010E949E
:10881000E9155C0181EE9CE00E94B6187C01F6012E
:1088200086819781FC01DF010D900020E9F7119707
:10883000AE1BBF0BBD010E94E9152D813E81020FC9
:10884000131FEF81F8850E0F1F1F020D131D040D5E
:10885000151D060D171D080D191D0A0D1B1D0E0DEA
:108860001F1D080F191FC8012896E2E10C944762EA
:10887000A8E2B0E0EEE3F4E40C943762082F11278D
:1088800007FD1095000F111FF801E95CFB4F859162
:108890009491F801E65AFE4F4591549139E0E32E48
:1088A000F12CEC0EFD1EB7010E94401CF801E15DA9
:1088B000FB4F859194919A838983F801E95FFB4F7F
:1088C000859194919C838B8381E28D838FE18E834C
:1088D000F886EF82CE0101960E94BD43A896E6E09D
:1088E0000C945362A8E1B0E0E8E7F4E40C9437623A
:1088F000E82EFF24E7FCF0948701000F111FF80118
:10890000EF55FC4F8591949101C0A895F999FDCF41
:108910000E943F639B01AC012F3F8FEF38078FEF21
:1089200048078FEF580759F4F701EE0FFF1FEE0FBE
:10893000FF1FE555FC4F2591359145915491F80164
:10894000EF50FC4F859194919A838983F801E95601
:10895000FC4F859194919C838B8382E18D838FE082
:108960008E83CA01B901AE01475F5F4F0E94463F47
:1089700098878F83CE0101960E94BD436896E6E0FA
:108980000C945362A0E0B0E0E8ECF4E40C943362A1
:108990005C0180E00E94DF426C0180E00E94724432
:1089A000EC0181E00E9472447C0182E00E947244EA
:1089B0008C0183E00E947244CC0DDD1DCE0DDF1DC5
:1089C000C00FD11FC80FD91F81E0A816B10419F438
:1089D0008BE193E002C083E593E00E94B618C80FD4
:1089E000D91F81E090E00E943D4260916405709142
:1089F0006505C80FD91F88E1AE010E943423CDB7A9
:108A0000DEB7EAE00C944F62AAE9B0E0EAE0F5E4F0
:108A10000C942B629C01880F991FBC01F3E0660F38
:108A2000771FFA95E1F7680F791F625C7A4F7093B0
:108A3000650560936405F901E659F84FE081E1307E
:108A400009F06EC6232B29F0E6E68E2EE6E09E2E78
:108A500004C076E6872E75E0972EC4016AE779E0B8
:108A60000E94B062FC01108261EDE62E67E0F62EF6
:108A700000E0F70165917491C40146E050E00E9466
:108A8000A262892B09F455C00F5F22E030E0E20EAC
:108A9000F31E063071F786E390E00E9484168CEE98
:108AA00091E00E94B6182C018EE999E00E94B61858
:108AB000480E591E882499248EE899E00E94B61821
:108AC0005C01F401EF52F84F859194910E94B61821
:108AD0008C018AE899E00E94B6186C01F401E55B0C
:108AE000F74F859194910E94B6187C0181E899E036
:108AF0000E94B6180A0D1B1D0C0D1D1D0E0D1F1D0D
:108B0000080F191F400E511E42E050E0840E951EC2
:108B10005CE08516910481F680E090E00E943D4281
:108B20006091640570916505480E591E88E1A201A7
:108B30000BC657E0452E512C480C591C002309F058
:108B400043C0D40117968C91882319F480E090E0FB
:108B500038C000E010E06E010894C11CD11C46E052
:108B6000842E912C800E911EF401E956FC4F6591E4
:108B70007491C2010E94B0627C01009701F10396DA
:108B8000B6010E94E23E813079F4F401EF55FC4FCA
:108B90008591949101C0A895F999FDCF49815A8199
:108BA0006B817C810E946D630894E108F108F701F4
:108BB000108202501040FFEF083F1F0781F681E04E
:108BC00090E00E94C244C2C5013009F081C0D201C8
:108BD0008C91882319F48824992459C0DE011C96AD
:108BE000EEE8F1E088E001900D928150E1F732E18A
:108BF000832E912C8C0E9D1E00E010E02CE3C22EE3
:108C0000D12CCC0EDD1E90E2B92E86E0282E312C20
:108C1000200E311EF101E95FFB4F65917491C20195
:108C20000E94B0627C01009779F1F6012B2D119220
:108C30002A95E9F7BC016D5F7F4FC6010E940B6367
:108C4000D4018D919C91B6010E940B63F101E95C06
:108C5000FB4F6591749101C0A895F999FDCFC601AC
:108C600040E250E00E944B630894E108F108F701EC
:108C70001082025010402EEF3FEF820E931E3FEF06
:108C8000083F130709F0C1CFB1E08B2E912C81E092
:108C90000E94DF426C0180E00E9438442C0181E098
:108CA0000E9438447C0182E00E9438448C0183E0B9
:108CB0000E9438444C0C5D1C4E0C5F1C400E511E33
:108CC000480E591E41E08416910409F07FC07BC014
:108CD000023009F08FC0D2018C91882319F48824C6
:108CE000992445C0C20167EB79E00E94B0627C0123
:108CF0000097D1F105960E94993D909317088093B3
:108D000016088F5F9F4F31F41092170810921608C3
:108D100001C0A895F999FDCF6091160870911708C8
:108D200084EC90E00E9479630894E108F108F7016F
:108D30001082C20164EB79E00E94B0620097A1F05A
:108D40000396BE016F5F7F4F0E94E23E813061F467
:108D500001C0A895F999FDCF49815A816B817C8129
:108D600080EC90E00E946D63A1E08A2E912C82E05D
:108D70000E94DF426C0184E00E9472442C018CEB63
:108D800099E00E94B6187C018E010C5E1F4F809105
:108D9000160890911708B8010E94F43CF801019060
:108DA0000020E9F73197E01BF10BC801BF010E94D9
:108DB000E9154C0C5D1C4E0C5F1C480E591EF1E071
:108DC0008F16910419F48BE193E002C083E593E0E0
:108DD0000E94B6187C01E40CF51C81E090E00E9432
:108DE0003D426091640570916505E80EF91E88E1C9
:108DF000A701AAC4033009F04FC1C2010E94164264
:108E0000813019F4F8E0FF2E05C0823011F40E9481
:108E10007C4FFF2483E00E94B6428C0189E29AE0F5
:108E20000E94B6186091640570916505080F191FBE
:108E300088E1A8010E943423882309F087C486E3CF
:108E400090E00E9484166F2CAA24BB24ECE22E2E04
:108E5000312C2C0E3D1E2F2D285FC656DF4F288348
:108E6000CA59D040E62DF0E074E0EE0FFF1F7A956E
:108E7000E1F7DE015C96E250F64F80E101900D9241
:108E80008150E1F7DBA04C8C5D8C3E8DCE57DF4FDF
:108E90003883C258D0404F8DCF57DF4F4883C158D9
:108EA000D04058A1C058DF4F5883C058D04079A057
:108EB000CAA08CA09DA08EA19FA1C258DF4F99830C
:108EC0008883CE57D04080E09BE00E94B6188C018A
:108ED0006394862D0E945A437C0186EF9AE00E949B
:108EE000B618E00EF11EE80EF91E8D2D815083306C
:108EF000D8F45E824D82CE57DF4F9881C258D04061
:108F00009F83CF57DF4FA881C158D040A887C05852
:108F1000DF4FB881C058D040B9877A86CB86CE0162
:108F200005960E946F4304C08FEE9AE00E94B61827
:108F3000E80EF91E85EE9AE00E94B6182701480E49
:108F4000591EE2E0DE1661F486ED9AE00E94B61842
:108F50007C0189EC9AE00E94B618E80EF91E77C0F1
:108F6000F1E0DF1609F06EC021E982162EE79206C5
:108F700044F08CEB9AE00E94B6187C01E40CF51CDE
:108F80005AC097FC02C08BE201C08DE20E94B2156C
:108F9000C40197FE03C0909581959F4FB1010E9437
:108FA000F43CF10101900020E9F73197E219F3094F
:108FB000C101BF010E94E9154C0187EB9AE00E94B4
:108FC000B6186C01C258DF4F48815981CE57D04046
:108FD00057FD02C08BE201C08DE20E94B215C2585B
:108FE000DF4F88819981CE57D04097FF03C090957D
:108FF00081959F4FB1010E94F43CF1010190002046
:10900000E9F7E219F3093397CE018E96BF010E946A
:10901000E9158C0183EB9AE00E94B61862E0E62E17
:10902000F12CE40CF51CE80CF91CEC0CFD1CE00E1A
:10903000F11EE80EF91E80EA9AE00E94B618E80ECA
:10904000F91E07C080E99AE00E94B6187C01E40C82
:10905000F51C85E89AE00E94B618E80EF91EAE0CE1
:10906000BF1CC656DF4F5881CA59D040651609F05B
:10907000F9CE609164057091650588E1A5010E94B3
:109080003423882309F062C386E390E00E948416AB
:1090900083E060E070E098C1043009F09DC1C20136
:1090A0000E941642813039F488E0C856DF4F888329
:1090B000C859D0400DC0823019F40E94714F03C0CE
:1090C000833009F4179AC856DF4F1882C859D04028
:1090D00084E00E94B6428C0188E29BE00E94B618B0
:1090E0006091640570916505080F191F88E1A8015A
:1090F0000E943423882309F029C386E390E00E946C
:109100008416C956DF4F1882C759D040EE961FAE5D
:109110001EAEEE9754E1252E312C2C0E3D1E8EEB0B
:109120009BE00E94B6188C01C956DF4FE881C759F1
:10913000D040C856DF4F9881C859D040E90FF0E0C1
:1091400044E0EE0FFF1F4A95E1F7CF018250954FA3
:10915000DC011C962D913D914D915C911F97CD5650
:10916000DF4F288339834A835B83C359D0401A96E3
:10917000CC901A971B96BC91C756DF4FB883C9593C
:10918000D040DF01AA5FB44FEC901196DC90DC0177
:1091900016966C91169715965C91DF01AE5FB44FF1
:1091A0007C91DC0113964C911397E050F54FE081D0
:1091B0002D913C9111971796FC90FF2009F4CAC09D
:1091C0008F2D8150843028F48AEA9BE00E94B618E3
:1091D0000BC03E832D83EF83488779875A876B873F
:1091E000CE0105960E946F43080F191F80EA9BE08D
:1091F0000E94B6182C01EF2DF0E0EE0FFF1FEE5A83
:10920000F84F859194910E94B618400E511E480E59
:10921000591EB5E0FB1609F03FC08AE99BE00E94A9
:10922000B6183C018E2D9D2DB1010E94603CF101CC
:1092300001900020E9F73197E219F309C101BF015C
:109240000E94E9154C0184E99BE00E94B6185C017C
:109250008C2DC756DF4F9881C959D040B1010E946B
:10926000603CF10101900020E9F73197E219F30920
:10927000C101BF010E94E9156C018DE89BE00E94CD
:10928000B6187C01CD56DF4F88819981C359D040F3
:10929000B1010E94603C41C0EAE0FE1621F0F7E017
:1092A000FF1609F05EC086E89BE00E94B6183C01FC
:1092B0008E2DB1010E94483CF10101900020E9F798
:1092C0003197E219F309C101BF010E94E9154C0170
:1092D0008FE79BE00E94B6185C018C2DB1010E94C3
:1092E000483CF10101900020E9F73197E219F309B8
:1092F000C101BF010E94E9156C0187E79BE00E9454
:10930000B6187C01CD56DF4F688179818A819B81B7
:10931000C359D040A1010E948A3CF1010190002074
:10932000E9F73197E219F309C101BF010E94E9157C
:109330008C0189E20E94B2150894411C511C460C14
:10934000571C480C591C4A0C5B1C4C0C5D1C4E0CE9
:109350005F1C05C081E69BE00E94B6182C01400E00
:10936000511E86E59BE00E94B618480E591EEE96E7
:109370002EAD3FADEE97240D351DEE963FAF2EAFCF
:10938000EE97C956DF4F3881C759D0403F5FC95665
:10939000DF4F3883C759D040383009F0C0CE6091D4
:1093A00064057091650588E1EE964EAD5FADEE9770
:1093B0000E943423882309F0C9C186E390E00E940B
:1093C000841684E061E070E00E9454428C0181E0E8
:1093D00090E00E943D4296C1053009F09CC185E0B5
:1093E0000E94B642CF56DF4F99838883C159D0403F
:1093F00086E89CE00E94B6188C0160912905709166
:109400002A0580912B0590912C052CE3E22EF12C5E
:10941000EC0EFD1EA7010E94463FBC018BE79CE0BD
:109420000E941C43CD57DF4F99838883C358D04097
:1094300060912D0570912E0580912F05909130053A
:10944000A7010E94463FBC018FE69CE00E941C439E
:10945000CB57DF4F99838883C558D0406091310541
:10946000709132058091330590913405A7010E94D7
:10947000463FBC018FE59CE00E941C43C957DF4F6B
:1094800099838883C758D0406091DD097091DE09C7
:109490008091DF099091E009A7010E94463FBC013D
:1094A00084E59CE00E941C43C757DF4F9983888363
:1094B000C958D04087E49CE06DEC79E00E941C43E1
:1094C000C557DF4F99838883CB58D0408091E409FA
:1094D000E82FF0E0EE0FFF1FED54F74F6591749108
:1094E000C7010E94926288E39CE0B7010E941C437E
:1094F000C357DF4F99838883CD58D04080917C013A
:10950000E82FF0E0EE0FFF1FE659F64F65917491DA
:10951000C7010E9492628CE29CE0B7010E941C434A
:10952000C157DF4F99838883CF58D0408091000185
:10953000B7010E94483C80910101BE01625C7F4FEF
:109540000E94483CB7016C5F7F4F809102010E94EE
:10955000483C8DE2FE01EE5BFF4F8083B701695FFF
:109560007F4F809103010E94483CB701675F7F4FA6
:10957000809104010E94483CB701655F7F4F809154
:1095800005010E94483CFE01E75BFF4F108280E22C
:109590009CE0B7010E941C431C0120919704822F7C
:1095A0006AE00E94CE61805D8CAF822F0E94CE6106
:1095B000905D9DAF1EAE8EE09CE0B7010E941C4303
:1095C0002C01C7016CE770E00E9492628DEF9BE076
:1095D000B7010E941C433C018090ED099090EE0978
:1095E000A090EF09B090F009C501B4012CE330E080
:1095F00040E050E00E941062CA01B901A7010E9438
:10960000733D7CE5C72ED12CCC0EDD1EB7016B5F00
:109610007F4FC6010E940B63C60167EF7BE00E948B
:109620007E62C501B4012CE330E040E050E00E94CE
:109630001062DC01CB01B7010E94F43CC601BE01FF
:10964000615C7F4F0E94EC62C60162EF7BE00E948A
:109650007E6283EE9BE0B6010E941C436C0186EDA6
:109660009BE00E94B6187C0181E090E00E943D42A0
:10967000CF56DF4F48815981C159D040040F151F83
:10968000CD57DF4FA881B981C358D0400A0F1B1FA7
:10969000CB57DF4FE881F981C558D0400E0F1F1F0F
:1096A000C957DF4F28813981C758D040020F131F97
:1096B000C757DF4F48815981C958D040040F151F43
:1096C000C557DF4FA881B981CB58D0400A0F1B1F67
:1096D000C357DF4FE881F981CD58D0400E0F1F1FCF
:1096E000C157DF4F28813981CF58D040020F131F57
:1096F000020D131D040D151D060D171D0C0D1D1D4E
:109700000E0D1F1D6091640570916505080F191FEE
:1097100088E1A80119C0609164057091650511C0C8
:10972000E23079F486E390E00E9484168BE791E0C2
:109730000E94B618AC01609164057091650588E1DE
:1097400003C081E140E050E00E943423C656DF4F61
:10975000E2E10C944762682F88E044E653E10E94FE
:10976000A31A0895E82FF0E0EE0FFF1FE85DFF4E0B
:109770004591549180E061E00E94A31A0895E82F7A
:10978000F0E0EE0FFF1FE558F04F4591549180E057
:1097900060E00E94A31A0895A0E1B0E0E2EDFBE4CE
:1097A0000C943562E090ED09F090EE090091EF091C
:1097B0001091F009C801B7012CE330E040E050E01F
:1097C0000E941062CA01B9016E010894C11CD11C2B
:1097D000A6010E94733D80E061E0AE014A5F5F4FE9
:1097E0000E94B31AC801B7012CE330E040E050E01A
:1097F0000E941062DC01CB01B6010E94F43C8AE0B9
:1098000061E0AE014C5F5F4F0E94B31A6096E8E0E2
:109810000C945162A4E0B0E0E0E1FCE40C9433620B
:10982000B82EA62E6A01FA0180817E010894E11CFF
:10983000F11CB7010E94D83C8E010E5F1F4F8B2D8B
:109840006A2DA8010E94B31A8AE30E944A1AF601FF
:109850008181B7010E94D83CC8010E94511A8AE355
:109860000E944A1AF6018281B7010E94D83CC801C1
:109870000E94511A2496EAE00C944F62A3E0B0E0F3
:10988000E4E4FCE40C943662D82E7A018B01403477
:109890008EE7580785E0680780E0780738F088E0B1
:1098A0006D2D4BE553E10E94A31A2EC0CB01BA01E6
:1098B00020E13EE040E050E00E9410622983C801B0
:1098C000B70120E13EE040E050E00E941062162F18
:1098D000072FF82EE92E2CE330E040E050E00E9404
:1098E00010622A83612F702F8F2D9E2D2CE330E084
:1098F00040E050E00E9410626B8388E06D2DAE0165
:109900004F5F5F4F0E940A4C2396E7E00C9452622F
:1099100080915408813049F440914D0850914E088F
:1099200060914F08709150081BC08731E1F480911D
:10993000490890914A08A0914B08B0914C088F5F5C
:109940009F4FAF4FBF4F19F4E8E6F0E115C04091CB
:10995000410850914208609143087091440881E0A9
:109960000E943E4C0895883119F4E6E6F0E104C007
:10997000893139F4E4E6F0E14591549188E061E001
:1099800004C088E061E044E653E10E94A31A089510
:10999000A3E2B0E0EEECFCE40C943262082F0E94EB
:1099A000721A093018F4402F4F5C02C0402F495002
:1099B0008FE060E00E94BE1AE02FF0E044E0EE0F7E
:1099C000FF1F4A95E1F7DE011496E250F54F80E162
:1099D00001900D928150E1F7DB849E81CF809884C5
:1099E000A984BA848D2D8150843068F18D2D8550E5
:1099F000823248F534E1E32EF12CEC0EFD1E892F66
:109A0000B7010E94D83C8E010B5E1F4F80E060E0E2
:109A1000A8010E94B31A8FE20E944A1A8C2DB70146
:109A20000E94D83CC8010E94511A80E20E944A1A42
:109A30009982AA82BB8286E060E0AE014F5F5F4FF1
:109A40000E940A4C06C080E060E040E453E10E94BE
:109A5000A31AED2DF0E0EE0FFF1FEE50FD4E4591E5
:109A6000549180E061E00E94A31AA396EBE00C946D
:109A70004E62A3E2B0E0EFE3FDE40C943162182FF4
:109A80000E94721A8BE00E94BF4BE12FF0E064E06D
:109A9000EE0FFF1F6A95E1F7DE011496E250F64FD4
:109AA00080E101900D928150E1F7DB84CE80BF8090
:109AB00088849984AA8454E1E52EF12CEC0EFD1ED5
:109AC000812F8F5FB7010E94D83C8E010B5E1F4F24
:109AD0008EE060E0A8010E94B31A80E061E00E947D
:109AE0007A1A8D2D8150823068F58C2DB7010E9435
:109AF000D83CC8010E94511A8FE20E944A1A8B2D4D
:109B0000B7010E94D83CC8010E94511A80E20E940D
:109B10004A1A89829A82AB8286E061E0AE014F5F89
:109B20005F4F0E940A4C80E20E944A1A82E0D816D7
:109B300011F482E404C081E0D81651F482E50E9459
:109B40004A1A06C080E061E040E453E10E94A31A93
:109B5000A396ECE00C944D62A3E1B0E0E2EBFDE4EF
:109B60000C942F628091F209E82FF0E0EE0FFF1FB6
:109B7000EE57FF4E65917491CE0108960E94926255
:109B800060902F017090310180903301A0903B01D3
:109B9000B0903C0100913701109138010F5F1F4FC9
:109BA000909035018091390190913A01FCE0CF2EDF
:109BB000D12CCC0EDD1E8459984FB6010E94F43C86
:109BC000EDE0EE2EF12CEC0EFD1E80E060E0A70132
:109BD0000E94B31A8FE20E944A1A802FB6010E9497
:109BE000D83CC7010E94511A8FE20E944A1A892D5F
:109BF000B6010E94D83CC7010E94511A80E20E941F
:109C00004A1A8E010C5F1F4FAA0CBB1CAA0CBB1C6E
:109C10008FE49EE0A80EB91EC801B5010E949262B1
:109C2000C8010E94511A80E20E944A1A8091E409F8
:109C3000882391F480910601803C11F481E415C0E1
:109C4000803411F489E411C0803811F484E40DC02B
:109C50008091F007805D09C0813011F482E505C074
:109C6000823011F08AE401C087E40E944A1A898296
:109C70007A826B8280E061E0AE014F5F5F4F0E94AD
:109C80000A4C80E20E944A1ACE0108960E94511A9C
:109C900080E20E944A1A8091E409823060F4809147
:109CA0000701BE016C5F7F4F0E94D83CCE01059634
:109CB0000E94511A1FC08230B9F48091E309877065
:109CC00011F48DE407C0813011F482E503C08230C5
:109CD00019F48AE50E944A1A8091E30983FF02C0C1
:109CE00082E506C086E404C080E30E944A1A81E34C
:109CF0000E944A1AE0917C01F0E0E559F14FE491AD
:109D00008E2F0E944A1A6396EEE00C944B62A0E1FB
:109D1000B0E0EDE8FEE40C9435620091E1090E94A8
:109D2000721A002319F40E94AC4DD7C0013019F506
:109D300080E060E041E40E94BE1A609129057091C4
:109D40002A0580912B0590912C058E010F5F1F4FE6
:109D5000A8010E94463F0E94511A80E061E04DE454
:109D60000E94BE1A60912D0570912E0580912F05DD
:109D70009091300524C0023041F580E060E047E476
:109D80000E94BE1A609131057091320580913305B1
:109D9000909134058E010F5F1F4FA8010E94463F2E
:109DA0000E94511A80E061E044E40E94BE1A609172
:109DB000DD097091DE098091DF099091E009A80129
:109DC0000E94463F0E94511A88C0033079F581E015
:109DD0000E94BF4B809197046AE00E94CE61805D33
:109DE0000E944A1A809197046AE00E94CE61892FEE
:109DF000805D0E944A1A83E00E94B24B04E0B0E00A
:109E0000EB2EB1E0FB2E6E010894C11CD11CF701B2
:109E100081917F01B6010E94483CAC01802F61E036
:109E20000E94B31A0E5F003191F757C0043061F4FD
:109E300080E060E04DEC59E00E94B31A84E00E949B
:109E4000B24B0E94884C49C0053089F586E00E94DB
:109E5000BF4B8091E409823031F0813021F0809154
:109E6000F309882391F188E060E044E653E10E9421
:109E7000A31A85E00E94B24B8091160890911708B2
:109E8000892B71F08091F4099091F509019741F4C3
:109E90000E94890EAB01BC0181E00E943E4C1DC0B6
:109EA00088E061E044E653E10E94A31A16C0063040
:109EB000A1F48CE00E94BF4B85E061E04FE453E1E8
:109EC0000E94A31A0E94CC4B08C00E94A40EAB01B2
:109ED000BC0180E00E943E4CCCCF6096E8E00C9440
:109EE000516280E091E0EEEFFAE0DF019C011D920B
:109EF00021503040E1F7089580E091E0EEEFF9E085
:109F0000DF019C011D9221503040E1F70895EF924E
:109F1000FF920F931F93182F8EE09BE06EEF7AE075
:109F200040EF50E00E94D3626091270170912801B8
:109F3000E0912501E0902301F090210100911F01A3
:109F4000F0911D01153079F44091910450919204E3
:109F500020918F043091900480918D0490918E0413
:109F6000A0E0B0E032C01A3011F0173089F48091CF
:109F70003805482F50E080913905282F30E0809136
:109F80003A0590913B05A0913C05B0913D051DC05F
:109F9000812F8850823048F080E090E0A0E0B0E06F
:109FA00020E030E040E050E010C04091AA04509121
:109FB000AB042091A8043091A9048091A004909151
:109FC000A104A091A204B091A30480930A0B9093E2
:109FD0000B0BA0930C0BB0930D0B3093090B20933C
:109FE000080B5093070B4093060B1093050BF0934F
:109FF000040B0093030BF092020BE092010BEF5F56
:10A00000E093000B6459784F7093FF0A6093FE0A47
:10A010001A3079F01B3169F0113259F01C3049F0D7
:10A020001D3039F0113029F0123019F0143009F0D8
:10A0300017981F910F91FF90EF900895FF920F9343
:10A040001F93F82E8EE09AE08C0100511040B80169
:10A0500040EF50E00E94D362809127019091280147
:10A060008459984F509125015F5FB0912301A091D1
:10A070002101F0911F01E0911D016091F2077091A3
:10A08000F3072091F4073091F5074091F107109202
:10A090000D0A10920C0A10920B0A40930A0AF092D1
:10A0A000050A3093090A2093080A7093070A6093FF
:10A0B000060AE093040AF093030AA093020AB093FD
:10A0C000010A5093000AF801918380831F910F9138
:10A0D000FF900895F8948091FE0B9091FF0B789477
:10A0E00020E0845690408B57934008F421E0822F63
:10A0F0000895CF93DF93EC011E860C960E94993D44
:10A100008E3391050CF069C09093660180936501D0
:10A110001C86CE010A960E94993D8C3391050CF065
:10A120005CC090936801809367011A86CE010896FF
:10A130000E94993D883191050CF04FC090936A01BF
:10A14000809369011886CE0106960E94993D00977A
:10A1500009F443C0803291050CF03FC090936C012C
:10A1600080936B011E82CE0104960E94993D019757
:10A170008C30910594F590936E0180936D011C8253
:10A18000CE010E94993D8C56974090937001809328
:10A190006F0110927201109271011092740110926D
:10A1A000730185E691E00E94321E97FF02C081E0B4
:10A1B00015C0F8946F5F7F4F8F4F9F4F60930D0CCA
:10A1C00070930E0C80930F0C9093100C10927D01E5
:10A1D00081E08093130C789401C080E0DF91CF91EF
:10A1E0000895AF92BF92CF92DF92EF92FF920F93BA
:10A1F0001F93379B08C01092F7091092F60987E069
:10A2000080937C0183C180917C01873019F482E0C6
:10A2100080937C011091F309112309F477C1113067
:10A22000D9F41092130C0E94841B8091F60990912E
:10A23000F709892B19F481E993E102C08AE893E1D7
:10A240000E94AD1C82E08093F3090E944B1B909307
:10A25000F9098093F8095AC11230D9F50E94981B68
:10A26000813009F03DC18091F6099091F709892B61
:10A27000C1F486E094E064E873E145E050E00E94B8
:10A28000A262892B39F481E090E09093F7098093E2
:10A29000F60911C080E490E00E94C10E10937C0189
:10A2A0001CC186E094E06BE773E148E050E00E9457
:10A2B000A262892B11F483E052C0A1E4B1E0EDE188
:10A2C000F1E082E101900D928150E1F71092F309E3
:10A2D0001EC1133041F40E94841B84E793E10E9465
:10A2E000AD1C84E0B0CF143009F051C00E94981B1F
:10A2F000813009F03FC0109210048EE094E00E947B
:10A30000993D009779F18032910564F590936C0145
:10A3100080936B0110920D048BE094E00E94993DB4
:10A3200001978C309105F4F490936E0180936D0148
:10A3300010920A0486E094E00E94993D8C56974062
:10A3400097FD10C09093700180936F01109272017D
:10A3500010927101109274011092730185E0809344
:10A36000F309D4C080E490E00E94C10E81E08093A4
:10A370007C01B3C00E944B1B2091F8093091F90970
:10A38000821B930B805D974008F4C0C0B4C01530A9
:10A3900041F40E94841B8DE693E10E94AD1C86E08F
:10A3A00052CF163009F0B2C00E94981B813009F0DC
:10A3B00097C010920E048CE094E00E94993D8C337B
:10A3C00091050CF08AC0909366018093650110920C
:10A3D0000B0489E094E00E94993D8C3391050CF0C8
:10A3E0007CC090936801809367011092080486E016
:10A3F00094E00E94993D883191050CF06EC09093D5
:10A400006A018093690185E691E00E94321E7B011A
:10A410008C0180E7A82E81E8B82E8FEFC82E8FEF31
:10A42000D82EEA0CFB1C0C1D1D1D17FD51C0F89405
:10A430002091000C3091010C4091020C5091030CC2
:10A44000789480911B0190911C01892B01F58091DA
:10A450001B0890911C080097D1F057016801A21ABF
:10A46000B30AC40AD50AA6019501D7FE07C05095C4
:10A470004095309521953F4F4F4F5F4FA0E0B0E0A2
:10A4800082179307A407B50714F482E022C0F8945A
:10A490000894E11CF11C011D111DE0920D0CF092BD
:10A4A0000E0C00930F0C1093100C10927D0182E0A3
:10A4B0008093130C78941092F5071092F407109281
:10A4C000F3071092F20710927C0110927B0105C0F5
:10A4D00081E080937C010E94A80B1092F30916C0C2
:10A4E0000E944B1B2091F8093091F909821B930BB4
:10A4F000805D974058F080E490E00E94C10E83E0B8
:10A5000080937C011092F30985E201C080E01F91E5
:10A510000F91FF90EF90DF90CF90BF90AF90089594
:10A52000A1E0B0E0E6E9F2E50C943162182F0E9458
:10A53000841B113019F482EE93E106C0123011F041
:10A54000CC244BC08EEA93E10E94AD1C0E944B1BB1
:10A550005C018C01CC24DD244E010894811C911CEB
:10A5600002C0DD2487010E944B1B7C0108171907DC
:10A5700009F0A895C7018A199B09805D974018F0DA
:10A5800025E2C22E2AC0DD2059F4C4010E94681BB6
:10A59000813041F78981843229F7DD24D394E2CFD9
:10A5A00081E0D81669F40E94981BC82E21E082171A
:10A5B00019F492E0D92ED6CF82E0C81699F60DC0D4
:10A5C00022E0D21679F686E094E060EA73E14DE08D
:10A5D00050E00E94A262892B21F68C2D2196ECE09E
:10A5E0000C944D62FC01808191819A3239F09A304D
:10A5F00029F03196992311F08927F6CF0E94483C23
:10A600000895A5E1B0E0E7E0F3E50C9438628091AD
:10A61000890490918A04892BD1F4CE0101960E947D
:10A62000681B813009F069C18981843209F065C1F4
:10A630000E944B1B909388048093870481E090E0F4
:10A6400090938A04809389041092860456C10E94D4
:10A65000981B813009F040C10091E30986E094E045
:10A66000BE016E5F7F4F0E94F25286E094E06AE284
:10A6700070E00E94F762FC0191818A81981731F4A1
:10A6800092818B81981711F410E001C014E20770D9
:10A69000023009F066C088E094E06CE973E143E0C1
:10A6A00050E00E94A262892B09F028C186E08093C5
:10A6B0007C0186E094E06CE270E00E94F762009713
:10A6C00091F08C010F5F1F4FCE010E96B80146E04E
:10A6D00050E00E942063C8016CE270E00E94F762C3
:10A6E0008C01009719F40E94A80BF4C00F5F1F4F54
:10A6F000CE010C96B80142E050E00E9420630D5F4D
:10A700001F4FCE010A96B80142E050E00E9420633C
:10A710000D5F1F4FCE010696B80144E050E00E9445
:10A720002063F8948091FE0B9091FF0B78948456EF
:10A7300090408B57934008F4E6C003C00E94A80BDA
:10A74000F1C08091120C882311F085E001C084E0F3
:10A7500080937C0110927B0110920C0C10920B0CD8
:10A76000CCC088E094E068E973E143E050E00E94E7
:10A77000A262892B09F0C2C086E094E06CE270E02E
:10A780000E94F762009709F4A5C08C010F5F1F4F6C
:10A79000CE010E96B80146E050E00E942063C80149
:10A7A0006CE270E00E94F762FC01009709F492C02D
:10A7B000F18001966CE270E00E94F762009709F464
:10A7C00089C001966CE270E00E94F762009709F47C
:10A7D00081C001966CE270E00E94F762009709F474
:10A7E00079C001966CE270E00E94F762009709F46C
:10A7F00071C001966CE270E00E94F762009709F464
:10A8000069C001966CE270E00E94F762009709F45B
:10A8100061C001966CE270E00E94F7628C010097C3
:10A8200009F458C0BC016F5F7F4FCE010C9642E027
:10A8300050E00E942063B8016D5F7F4FCE010A9601
:10A8400042E050E00E942063B8016B5F7F4FCE0171
:10A85000089642E050E00E942063F801858187332A
:10A8600024F081E38E8389E303C082E38E8380E357
:10A870008F83F8948091FE0B9091FF0B789484560F
:10A8800090408B57934008F446C021E4F21661F4DF
:10A890008091120C882311F085E001C084E0809340
:10A8A0007C0110927B0110C086E5F81611F013E2CE
:10A8B0000CC086E080937C018091EB099091EC09BB
:10A8C000892B79F30E94A80B10E010920C0C1092C7
:10A8D0000B0C14C013E212C00E944B1B2091870482
:10A8E00030918804821B930B885E934030F0109265
:10A8F0008A041092890415E201C010E0812F659648
:10A90000E5E00C945462CE0106960E9479508823AB
:10A9100009F017CF13CFCE0106960E9479508823F5
:10A9200009F0B3CF12E2EACFA8E0B0E0EAE9F4E53B
:10A930000C94376281E00E949D1A81E061E046ED4F
:10A9400056E10E94A31A8091EB099091EC097E01D7
:10A950000894E11CF11CB7010E94F43CAC0186E0B4
:10A9600061E00E94B31A86E061E0A70125E000E003
:10A9700010E00E941340892B19F421E030E012C04E
:10A98000C7010E94993DBC019093EC098093EB09AB
:10A9900001C0A895F999FDCF82ED90E00E947963FE
:10A9A00020E030E0C9012896E6E00C945362A8E06C
:10A9B000B0E0EDEDF4E50C94376281E00E949D1A61
:10A9C00081E061E044EE56E10E94A31A8091E9091A
:10A9D0009091EA097E010894E11CF11CB7010E94E4
:10A9E000F43CAC0186E061E00E94B31A86E061E0CD
:10A9F000A70125E000E010E00E941340892B19F424
:10AA000021E030E012C0C7010E94993DBC01909343
:10AA1000EA098093E90901C0A895F999FDCF80ED75
:10AA200090E00E94796320E030E0C9012896E6E0DA
:10AA30000C9453621F93182F0E94721AE12FF0E0BA
:10AA4000EE0FFF1FEF5DFA4E4591549180E060E0FC
:10AA50000E94A31A1F910895EF92FF921F93DF9314
:10AA6000CF930F92CDB7DEB780E10E941A551091B7
:10AA7000FD09E12FF0E0EE0FFF1FEF54F94E459175
:10AA8000549180E061E00E94A31A7E010894E11CC9
:10AA9000F11C812F63E0A7010E94F03F182F8981EC
:10AAA000893159F18431C9F41093FD0901C0A89589
:10AAB000F999FDCF8CE390E00E944563682F01C0B7
:10AAC000A895F999FDCF9C7F192B8CE390E0712F0D
:10AAD0000E94796320E030E012C081E00E949D1A5C
:10AAE000E12FF0E0EE0FFF1FEF54F94E4591549126
:10AAF00080E061E00E94A31ACCCF21E030E0C901E0
:10AB00000F90CF91DF911F91FF90EF900895EF92FA
:10AB1000FF921F93DF93CF930F92CDB7DEB78FE0F5
:10AB20000E941A5510918B04E12FF0E0EE0FFF1FE9
:10AB3000EA58F94E4591549180E061E00E94A31AD1
:10AB40007E010894E11CF11C812F67E0A7010E949F
:10AB5000F03F182F8981893109F45BC0843109F0F5
:10AB600048C010938B048091E409823079F51092EB
:10AB7000C100112319F484E395E01DC0113019F4CC
:10AB80008AE992E018C0123019F48CE491E013C005
:10AB9000133019F485EA90E00EC0143019F482E500
:10ABA00090E009C0153019F489E290E004C0163035
:10ABB00031F48BE190E09093C5008093C40088E964
:10ABC0008093C1008091C60001C0A895F999FDCF7E
:10ABD00086E090E00E944563792F01C0A895F9991D
:10ABE000FDCF86E090E0612F0E94796320E030E0A5
:10ABF00012C081E00E949D1AE12FF0E0EE0FFF1FCE
:10AC0000EA58F94E4591549180E061E00E94A31A00
:10AC10009BCF21E030E0C9010F90CF91DF911F91D0
:10AC2000FF90EF900895A8E0B0E0E9E1F6E50C941C
:10AC300037628EE00E941A5581E061E047EB56E1F1
:10AC40000E94A31A80911B0890911C087E01089411
:10AC5000E11CF11CB7010E94F43CAC0187E061E00B
:10AC60000E94B31A87E061E0A70125E000E010E050
:10AC70000E941340892B19F421E030E012C0C70173
:10AC80000E94993DBC0190931C0880931B0801C051
:10AC9000A895F999FDCF88EC90E00E94796320E0B7
:10ACA00030E0C9012896E6E00C945362A8E0B0E0D9
:10ACB000ECE5F6E50C9437628DE00E941A5581E0D0
:10ACC00061E046EC56E10E94A31A8091140890912D
:10ACD00015087E010894E11CF11CB7010E94F43CA8
:10ACE000AC0189E061E00E94B31A89E061E0A7014C
:10ACF00025E000E010E00E941340892B19F421E0C8
:10AD000030E012C0C7010E94993DBC019093150824
:10AD10008093140801C0A895F999FDCF86EC90E0C6
:10AD20000E94796320E030E0C9012896E6E00C94A7
:10AD30005362EF92FF921F93DF93CF930F92CDB7A1
:10AD4000DEB78CE00E941A558091E30990E073E031
:10AD5000969587957A95E1F7182F1170E12FF0E01D
:10AD6000EE0FFF1FED5FF94E4591549180E061E0D9
:10AD70000E94A31A7E010894E11CF11C812F62E05D
:10AD8000A7010E94F03F182F89818931A1F18431F8
:10AD900011F501C0A895F999FDCF8CE390E00E94D0
:10ADA00045632091E309112331F4277F2093E309C0
:10ADB000BC01677F07C028602093E309BC0168607D
:10ADC00001C0A895F999FDCF8CE390E00E947963CA
:10ADD00020E030E012C081E00E949D1AE12FF0E0F7
:10ADE000EE0FFF1FED5FF94E4591549180E061E059
:10ADF0000E94A31AC3CF21E030E0C9010F90CF9188
:10AE0000DF911F91FF90EF900895EF92FF921F93B3
:10AE1000DF93CF930F92CDB7DEB78BE00E941A5528
:10AE20001091E3091770E12FF0E0EE0FFF1FE751DB
:10AE3000FA4E4591549180E061E00E94A31A7E0190
:10AE40000894E11CF11C812F63E0A7010E94F03FF0
:10AE5000182F8981893109F439C0843139F501C04D
:10AE6000A895F999FDCF8CE390E00E944563BC0161
:10AE7000687F8091E309887F8093E309113029F48A
:10AE800081608093E309616008C0123031F4826010
:10AE90008093E309626001C0A895F999FDCF8CE326
:10AEA00090E00E94796320E030E012C081E00E94CF
:10AEB0009D1AE12FF0E0EE0FFF1FE751FA4E45918A
:10AEC000549180E061E00E94A31ABDCF21E030E000
:10AED000C9010F90CF91DF911F91FF90EF900895DE
:10AEE000CF92DF92FF920F931F93DF93CF930F9236
:10AEF000CDB7DEB788E00E941A55F090F209EF2D29
:10AF0000F0E0EE0FFF1FE756FA4E4591549180E0B6
:10AF100061E00E94A31A6E010894C11CD11C8F2D00
:10AF200066E0A6010E94F03FF82E8981893109F47C
:10AF300034C00F2D10E0843109F5F092F209F801C8
:10AF4000EE0FFF1FEE0FFF1FEB55FA4E8591959107
:10AF5000A591B4918093770190937801A0937901A2
:10AF6000B0937A0101C0A895F999FDCF8CEC90E0DF
:10AF7000B8010E94796320E030E011C081E00E94B6
:10AF80009D1AF801EE0FFF1FE756FA4E45915491B6
:10AF900080E061E00E94A31AC2CF21E030E0C90145
:10AFA0000F90CF91DF911F910F91FF90DF90CF9085
:10AFB0000895CF92DF92FF920F931F93DF93CF9369
:10AFC0000F92CDB7DEB787E00E941A5501C0A89551
:10AFD000F999FDCF8AEC90E00E9445638C01FF2433
:10AFE000F394F822EF2DF0E0EE0FFF1FED5CF94E29
:10AFF0004591549180E061E00E94A31A6E0108948B
:10B00000C11CD11C8F2D62E0A6010E94F03FF82EDA
:10B010008981893181F18431F1F48091E409FF2043
:10B0200039F4B8016E7F813061F41092E40909C0EF
:10B03000B8016160882329F481E08093E40901C0AC
:10B04000A895F999FDCF7F778AEC90E00E9479630B
:10B0500020E030E012C081E00E949D1AEF2DF0E068
:10B06000EE0FFF1FED5CF94E4591549180E061E0D9
:10B070000E94A31AC7CF21E030E0C9010F90CF9101
:10B08000DF911F910F91FF90DF90CF900895A8E07E
:10B09000B0E0EDE4F8E50C94376286E00E941A55C2
:10B0A00080E061E042EF56E10E94A31A8091160809
:10B0B000909117087E010894E11CF11CB7010E94D1
:10B0C000F43CAC0189E061E00E94B31A89E061E0E0
:10B0D000A70125E000E010E00E941340892B19F43D
:10B0E00021E030E012C0C7010E94993DBC0190935D
:10B0F00017088093160801C0A895F999FDCF84EC34
:10B1000090E00E94796320E030E0C9012896E6E0F3
:10B110000C945362A4E1B0E0E0E9F8E50C943562E8
:10B120006B010E941A5501C0A895F999FDCFC6017F
:10B130000E943F6369837A838B839C8345E0E42E7E
:10B14000F12CEC0EFD1EA7010E94463F81E061E05C
:10B15000A7012FE000E010E00E941340892B19F4B2
:10B1600021E030E015C0C701BE016F5F7F4F0E9434
:10B17000E23E813059F401C0A895F999FDCF49818B
:10B180005A816B817C81C6010E946D6320E030E0B2
:10B19000C9016496E8E00C94516285E060EC70E0CF
:10B1A0000E948A58089583E06CE270E00E948A58F9
:10B1B000089582E068E270E00E948A58089581E074
:10B1C00064E270E00E948A58089580E060E270E0D6
:10B1D0000E948A580895CF92DF92FF920F931F9397
:10B1E000DF93CF930F92CDB7DEB784E00E941A555C
:10B1F00001C0A895F999FDCF8CE090E00E944563CD
:10B200008C01F12EFF1CFF24FF1CEF2DF0E0EE0F50
:10B21000FF1FEA5EF94E4591549180E061E00E9483
:10B22000A31A6E010894C11CD11C8F2D62E0A601E7
:10B230000E94F03FF82E8981893141F18431B1F4C7
:10B24000FF2029F410925408B8017F7706C080933C
:10B250005408B801706801C0A895F999FDCF8CE039
:10B2600090E00E94796320E030E012C081E00E940B
:10B270009D1AEF2DF0E0EE0FFF1FEA5EF94E4591AB
:10B28000549180E061E00E94A31ACFCF21E030E02A
:10B29000C9010F90CF91DF911F910F91FF90DF9027
:10B2A000CF900895A4E0B0E0E8E5F9E50C943A62A7
:10B2B000182F0E94721A80E060E046E057E10E9479
:10B2C000A31AE12FFF27E7FDF095EE0FFF1FEF5DBB
:10B2D000FA4E4591549180E061E00E94A31A812FBB
:10B2E0008F5FBE016F5F7F4F0E94D83C8BE060E0B4
:10B2F000AE014E5F5F4F0E94B31A8DE060E042E006
:10B3000057E10E94A31A2496E3E00C945662CF9270
:10B31000DF92FF920F931F93DF93CF93CDB7DEB7EA
:10B32000A3970FB6F894DEBF0FBECDBFDE01129615
:10B33000E6E9F1E082E201900D928150E1F70E948E
:10B340005259FF246E010894C11CD11C8F2D62E15B
:10B35000A6010E94F03FF82E89818931C1F0843125
:10B3600019F000E010E00EC081E1F81681F0EF2D39
:10B37000F0E0EE0FFF1FEC0DFD1D0180F281E02DCE
:10B3800009958C018F2D0E945259012BF9F2809161
:10B390005408882309F045C01092560810925508A9
:10B3A00080E290E044E651E068EA70EC0E94861C7E
:10B3B0006093290570932A0580932B0590932C05A3
:10B3C00084E290E040E05FEF6FEF7FEF0E94861C29
:10B3D00060932D0570932E0580932F059093300573
:10B3E00088E290E041E051E068EA70EC0E94861C3F
:10B3F0006093310570933205809333059093340543
:10B400008CE290E041E051E068EA70EC0E94861C1A
:10B410006093DD097093DE098093DF099093E00962
:10B4200017C08431A9F481E090E09093560880938E
:10B430005508A8E0B1E0EDE1F1E082E101900D9264
:10B440008150E1F70E94AB28882311F00E94874FBA
:10B45000A3960FB6F894DEBF0FBECDBFCF91DF919C
:10B460001F910F91FF90DF90CF900895EF92FF9280
:10B470000F93DF93CF93CDB7DEB760970FB6F894F5
:10B48000DEBF0FBECDBFA82F002309F461C07E012F
:10B490000894E11CF11C88E0F70111928A95E9F704
:10B4A00029833A834B835C836D837E83AF83988744
:10B4B00080E2801BE82FFF27E7FDF09549815A8144
:10B4C0006B817C81181684F019861A861B861C866F
:10B4D000882799278E1B9F0B04C0440F551F661F9A
:10B4E000771F8A95D2F728C0202F332727FD309564
:10B4F000DB01CA01022E04C0880F991FAA1FBB1FBF
:10B500000A94D2F789879A87AB87BC8704C076955F
:10B51000679557954795EA95D2F78D819E81AF81C2
:10B52000B88504C0880F991FAA1FBB1F2A95D2F7A0
:10B53000482B592B6A2B7B2B4D875E876F87788B27
:10B5400029853A854B855C856D857E85AF85988993
:10B550008A2F60960FB6F894DEBF0FBECDBFCF9195
:10B56000DF910F91FF90EF900895EF92FF920F936C
:10B57000DF93CF93CDB7DEB760970FB6F894DEBFF9
:10B580000FBECDBFA82F002309F467C07E01089429
:10B59000E11CF11C88E0F70111928A95E9F72983F3
:10B5A0003A834B835C836D837E83AF83988780E28D
:10B5B000801B4D815E816F817885E82FFF27E7FD35
:10B5C000F0951816B4F0DB01CA01BB0F880B982F59
:10B5D000DC018D879E87AF87B88B882799278E1BC4
:10B5E0009F0B04C075956795579547958A95D2F737
:10B5F00028C0202F332727FD3095DB01CA01022EFA
:10B6000004C0B595A795979587950A94D2F78D872D
:10B610009E87AF87B88B04C0440F551F661F771FE6
:10B62000EA95D2F789819A81AB81BC8104C0B69535
:10B63000A795979587952A95D2F7482B592B6A2B72
:10B640007B2B49875A876B877C8729853A854B8571
:10B650005C856D857E85AF8598898A2F60960FB64B
:10B66000F894DEBF0FBECDBFCF91DF910F91FF9059
:10B67000EF900895AEE5B0E0E0E4FBE50C942B62BA
:10B68000A8E04E010894811C911CF4016A2E1192CD
:10B690006A94E9F729833A834B835C836D837E83C5
:10B6A0008F839887CE010996FC011192AA95E9F73C
:10B6B000A986BA86CB86DC86ED86FE860F87188B38
:10B6C00029843A844B845C84ED84FE840F85188938
:10B6D00069807A808B809C806DA67EA68FA698AAB2
:10B6E0006D807E808F809884E114F104010511053E
:10B6F00009F0B3C3621473048404950408F03DC1D7
:10B7000000E0201600E0300601E0400600E05006B0
:10B7100088F41FEF211631044104510439F030F050
:10B7200048E0E42EF12C012D112D18C0EE24FF2449
:10B73000870114C020E0221620E0320620E04206F5
:10B7400021E0520630F038E1E32EF12C012D112DCD
:10B7500005C020E1E22EF12C012D112DD201C101F5
:10B760000E2C04C0B695A795979587950A94D2F7A5
:10B7700088549E4FDC012C9180E290E0A0E0B0E084
:10B780008E199F09A00BB10B7C018D01E21AF10803
:10B7900001091109E114F10401051105A1F10E2CB3
:10B7A00004C0220C331C441C551C0A94D2F7A4017B
:10B7B00093010E2C04C0220F331F441F551F0A94FF
:10B7C000D2F780E290E08E199F096DA47EA48FA429
:10B7D00098A804C096948794779467948A95D2F732
:10B7E000622A732A842A952AADA4BEA4CFA4D8A81D
:10B7F00004C0AA0CBB1CCC1CDD1CEA94D2F7ADA67D
:10B80000BEA6CFA6D8AA6201EE24FF24CDAADEAA46
:10B81000EFAAF8AE920181012070307009AF1AAF23
:10B820002BAF3CAFC401B301A70196010E94EE61AA
:10B830007B018C01C401B3012DA93EA94FA958ADCC
:10B840000E94EE61C901DA013C014D01C401B3015E
:10B8500029AD3AAD4BAD5CAD0E94AF619B01AC012F
:10B860008701FF24EE24ADA4BEA4CFA4D8A8C601AE
:10B87000AA27BB2757016801A82AB92ACA2ADB2AA6
:10B88000A216B306C406D506E0F408946108710850
:10B8900081089108A20CB31CC41CD51CA214B304CB
:10B8A000C404D50470F0A216B306C406D50648F445
:10B8B00008946108710881089108A20CB31CC41C8B
:10B8C000D51CA21AB30AC40AD50AC601B5012DA90E
:10B8D0003EA94FA958AD0E94EE617B018C01C601C3
:10B8E000B5012DA93EA94FA958AD0E94EE61C9012D
:10B8F000DA015C016D01C601B50129AD3AAD4BAD70
:10B900005CAD0E94AF619B01AC018701FF24EE2476
:10B910008DA59EA5AFA5B8A9A070B070E82AF92A98
:10B920000A2B1B2BE216F30604071507C0F4089434
:10B93000A108B108C108D108E20CF31C041D151DB3
:10B94000E214F3040405150550F0E216F3060407AB
:10B95000150728F40894A108B108C108D108D3013B
:10B960009927882786017501E82AF92A0A2B1B2BBB
:10B97000E9AAFAAA0BAB1CABCFC4211431044104D1
:10B98000510471F461E070E080E090E020E030E08C
:10B9900040E050E00E94EE61C901DA011C012D0176
:10B9A00000E0201600E0300601E0400600E050060E
:10B9B00088F41FEF211631044104510431F028F0BE
:10B9C00048E050E060E070E017C040E050E060E028
:10B9D00070E012C020E0221620E0320620E042068D
:10B9E00021E0520628F048E150E060E070E004C039
:10B9F00040E150E060E070E0D201C101042E04C0DB
:10BA0000B695A795979587950A94D2F788549E4F37
:10BA1000DC012C91E0E2EE2EF12C012D112DD8014C
:10BA2000C701841B950BA60BB70B821B9109A109BB
:10BA3000B1090097A105B10561F464015301A21891
:10BA4000B308C408D50831E0632E712C812C912CE9
:10BA50001EC16F968FAF6F97082E04C0220C331C47
:10BA6000441C551C0A94D2F7EE2DE81B64015301C7
:10BA70000E2E04C0D694C794B794A7940A94D2F714
:10BA8000A40193016F960FAC6F9704C0220F331F70
:10BA9000441F551F0A94D2F76DA47EA48FA498A8C2
:10BAA0000E2E04C096948794779467940A94D2F7E4
:10BAB00084017301E22AF32A042B152BE9A6FAA6C6
:10BAC0000BA71CA7320188249924920181012070C0
:10BAD000307021960CAF1DAF2EAF3FAF2197C6013E
:10BAE000B501A40193010E94EE617B018C01C601A6
:10BAF000B501A40193010E94EE61C901DA01259606
:10BB00008CAF9DAFAEAFBFAF2597BC01CD012196E5
:10BB10002CAD3DAD4EAD5FAD21970E94AF619B0155
:10BB2000AC018701FF24EE24A9A4BAA4CBA4DCA411
:10BB3000C601AA27BB275C016D01AE28BF28C02A19
:10BB4000D12AA216B306C406D50660F525966CADBB
:10BB50007DAD8EAD9FAD2597615070408040904087
:10BB600025966CAF7DAF8EAF9FAF2597A20CB31C0F
:10BB7000C41CD51CA214B304C404D50498F0A216A6
:10BB8000B306C406D50670F4615070408040904002
:10BB900025966CAF7DAF8EAF9FAF2597A20CB31CDF
:10BBA000C41CD51CA21AB30AC40AD50AC601B50121
:10BBB000A40193010E94EE617B018C01C601B501D5
:10BBC000A40193010E94EE61C901DA013C014D011B
:10BBD000C401B30121962CAD3DAD4EAD5FAD2197B3
:10BBE0000E94AF619B01AC018701FF24EE2489A56F
:10BBF0009AA5ABA5BCA5A070B07057016801A82A92
:10BC0000B92ACA2ADB2AA216B306C406D506E0F46E
:10BC100008946108710881089108A20CB31CC41C27
:10BC2000D51CA214B304C404D50470F0A216B30644
:10BC3000C406D50648F40894610871088108910883
:10BC4000A20CB31CC41CD51C8DA59EA5AFA5B8A97C
:10BC50006F960FAC6F9704C0880F991FAA1FBB1F68
:10BC60000A94D2F78DA79EA7AFA7B8ABA21AB30AC2
:10BC7000C40AD50A2596ECACFDAC0EAD1FAD2597D8
:10BC8000D70199278827682A792A8A2A9B2A82013C
:10BC90002227332729960CAF1DAF2EAF3FAF299730
:10BCA000A2019101407050702D962CAF3DAF4EAF68
:10BCB0005FAF2D97C601B50129962CAD3DAD4EADB8
:10BCC0005FAD29970E94EE617B018C01C601B50131
:10BCD00029962CAD3DAD4EAD5FAD29970E94EE612A
:10BCE000C901DA0161968CAF9DAFAEAFBFAF61976E
:10BCF000BC01CD012D962CAD3DAD4EAD5FAD2D9768
:10BD00000E94AF619B01AC018701FF24EE24ADA42A
:10BD1000BEA4CFA4D8A8C601AA27BB275701680193
:10BD2000A82AB92ACA2ADB2AA216B306C406D5064F
:10BD300060F561966CAD7DAD8EAD9FAD6197615044
:10BD400070408040904061966CAF7DAF8EAF9FAFEA
:10BD50006197A20CB31CC41CD51CA214B304C40468
:10BD6000D50498F0A216B306C406D50670F4615047
:10BD700070408040904061966CAF7DAF8EAF9FAFBA
:10BD80006197A20CB31CC41CD51CA21AB30AC40A26
:10BD9000D50AC601B50129962CAD3DAD4EAD5FADBE
:10BDA00029970E94EE617B018C01C601B50129969D
:10BDB0002CAD3DAD4EAD5FAD29970E94EE61C9013E
:10BDC000DA015C016D01C601B5012D962CAD3DADCA
:10BDD0004EAD5FAD2D970E94AF619B01AC01870115
:10BDE000FF24EE248DA59EA5AFA5B8A9A070B070C4
:10BDF000E82AF92A0A2B1B2BE216F306040715077B
:10BE0000C0F40894A108B108C108D108E20CF31CE1
:10BE1000041D151DE214F3040405150550F0E21687
:10BE2000F3060407150728F40894A108B108C1080F
:10BE3000D1086196ECACFDAC0EAD1FAD6197D7019A
:10BE40009927882796018501082B192B2A2B3B2B34
:10BE500009AB1AAB2BAB3CAB62C26E147F048006FD
:10BE6000910608F451C220E0E21620E0F20621E03B
:10BE7000020720E0120788F43FEFE316F104010502
:10BE8000110531F028F048E050E060E070E017C0A4
:10BE900040E050E060E070E012C040E0E41640E0B6
:10BEA000F40640E0040741E0140728F048E150E0C0
:10BEB00060E070E004C040E150E060E070E0D80174
:10BEC000C701042E04C0B695A795979587950A9447
:10BED000D2F788549E4FDC012C9130E2A32EB12C76
:10BEE000C12CD12CD601C501841B950BA60BB70B19
:10BEF000821B9109A109B1090097A105B10589F437
:10BF0000E614F7040805190508F4F2C16DA47EA42F
:10BF10008FA498A8621473048404950408F0E8C1FF
:10BF2000F3C16E968FAF6E97082E04C0EE0CFF1C07
:10BF3000001F111F0A94D2F76A2D681BD201C1019C
:10BF4000062E04C0B695A795979587950A94D2F7C3
:10BF50005C016D01AE28BF28C02AD12AADA2BEA2C5
:10BF6000CFA2D8A6720161016E960FAC6E9704C085
:10BF7000CC0CDD1CEE1CFF1C0A94D2F7C9A2DAA27D
:10BF8000EBA2FCA264015301062E04C0D694C79410
:10BF9000B794A7940A94D2F7D401C3016E960FAC5C
:10BFA0006E9704C0880F991FAA1FBB1F0A94D2F76F
:10BFB000EDA4FEA40FA518A904C016950795F79443
:10BFC000E7946A95D2F737014801682A792A8A2AC4
:10BFD0009B2A6D8E7E8E8F8E98A2EDA0FEA00FA163
:10BFE00018A53801882499249801870120703070A1
:10BFF00065960CAF1DAF2EAF3FAF6597C601B5017B
:10C00000A40193010E94EE617B018C01C601B50180
:10C01000A40193010E94EE61C901DA011C012D0106
:10C02000C201B10165962CAD3DAD4EAD5FAD6597DA
:10C030000E94AF619B01AC018701FF24EE24AD8C0F
:10C04000BE8CCF8CD8A0C601AA27BB275701680198
:10C05000A82AB92ACA2ADB2AA216B306C406D5061C
:10C0600000F508942108310841085108EDA0FEA010
:10C070000FA118A5AE0CBF1CC01ED11EAE14BF046C
:10C08000C006D10670F0A216B306C406D50648F461
:10C0900008942108310841085108AE0CBF1CC01E8D
:10C0A000D11EA21AB30AC40AD50AC601B501A40159
:10C0B00093010E94EE617B018C01C601B501A401D0
:10C0C00093010E94EE61C901DA013C014D01C401F6
:10C0D000B30165962CAD3DAD4EAD5FAD65970E9449
:10C0E000AF619B01AC018701FF24EE248D8D9E8DF5
:10C0F000AF8DB8A1A070B07057016801A82AB92A05
:10C10000CA2ADB2AA216B306C406D50600F508948F
:10C1100061087108810891086DA17EA18FA198A581
:10C12000A60EB71EC81ED91EA616B706C806D90683
:10C1300070F0A216B306C406D50648F40894610848
:10C14000710881089108A60EB71EC81ED91ED60117
:10C15000C501821B930BA40BB50B898F9A8FAB8FF4
:10C16000BC8FD1019927882764015301A82AB92AD5
:10C17000CA2ADB2AA9AABAAACBAADCAA8601750117
:10C180002FEF3FEF40E050E0E222F322042315239B
:10C19000A601662777276D964CAF5DAF6EAF7FAF78
:10C1A0006D97A9A0BAA0CBA0DCA06FEF7FEF80E0D5
:10C1B00090E0A622B722C822D92289A19AA1ABA1D8
:10C1C000BCA11D0144245524C801B701A601950155
:10C1D0000E94AF6169966CAF7DAF8EAF9FAF6997DC
:10C1E000C801B701A20191010E94AF613B014C015E
:10C1F0006D966CAD7DAD8EAD9FAD6D97A601950131
:10C200000E94AF617B018C016D966CAD7DAD8EADF2
:10C210009FAD6D97A20191010E94AF615B016C011E
:10C22000A8019701260D371D481D591D69966CAC54
:10C230007DAC8EAC9FAC6997C401AA27BB27280FA1
:10C24000391F4A1F5B1F2E153F054007510748F451
:10C25000E12CF12C61E0062F112DAE0CBF1CC01E8D
:10C26000D11ECA01AA27BB27BC01CD016A0D7B1DC7
:10C270008C1D9D1D698C7A8C8B8C9C8C6616770628
:10C280008806990640F1661577058805990509F035
:10C2900043C0D9019927882769962CAD3DAD4EAD95
:10C2A0005FAD699740705070820F931FA41FB51F38
:10C2B0002DA53EA54FA558A96E960FAC6E9704C04C
:10C2C000220F331F441F551F0A94D2F7281739072E
:10C2D0004A075B0708F509A91AA92BA93CA901502F
:10C2E00010402040304009AB1AAB2BAB3CAB14C024
:10C2F00066247724430121E030E040E050E029ABA0
:10C300003AAB4BAB5CAB0BC066247724430119AA54
:10C310001AAA1BAA1CAA03C0662477244301FE01A3
:10C32000719688E0DF011D928A95E9F7A9A8BAA85D
:10C33000CBA8DCA8A98ABA8ACB8ADC8A6D8A7E8AD5
:10C340008F8A988E29A93A894B895C89662D7E89C6
:10C350008F89988DC25ADF4FE2E10C944762629F49
:10C36000D001739FF001829FE00DF11D649FE00DED
:10C37000F11D929FF00D839FF00D749FF00D659F4E
:10C38000F00D9927729FB00DE11DF91F639FB00D4D
:10C39000E11DF91FBD01CF0111240895991B79E01A
:10C3A00004C0991F961708F0961B881F7A95C9F745
:10C3B00080950895AA1BBB1B51E107C0AA1FBB1F94
:10C3C000A617B70710F0A61BB70B881F991F5A9521
:10C3D000A9F780959095BC01CD010895A1E21A2E90
:10C3E000AA1BBB1BFD010DC0AA1FBB1FEE1FFF1F19
:10C3F000A217B307E407F50720F0A21BB30BE40B69
:10C40000F50B661F771F881F991F1A9469F76095AF
:10C410007095809590959B01AC01BD01CF01089569
:10C4200097FB092E05260ED057FD04D0D7DF0AD082
:10C43000001C38F450954095309521953F4F4F4F53
:10C440005F4F0895F6F790958095709561957F4FB1
:10C450008F4F9F4F08952F923F924F925F926F920E
:10C460007F928F929F92AF92BF92CF92DF92EF9284
:10C47000FF920F931F93CF93DF93CDB7DEB7CA1B05
:10C48000DB0B0FB6F894DEBF0FBECDBF09942A8830
:10C49000398848885F846E847D848C849B84AA84D8
:10C4A000B984C884DF80EE80FD800C811B81AA8165
:10C4B000B981CE0FD11D0FB6F894DEBF0FBECDBF30
:10C4C000ED010895911106C080538A5010F0865CEA
:10C4D00006C0089599278827089585FDFBCF8062BF
:10C4E0009111F8CF81568A51E0F70895911108957E
:10C4F00081568A5108F4805285580895FB01DC0169
:10C500000D900020E9F7119705900D920020E1F7BA
:10C510000895FB01DC018D91059080190110D9F37C
:10C52000990B0895FB01DC0105900D920020E1F7C5
:10C530000895FC0105900020E9F7809590958E0FF5
:10C540009F1F0895FB01DC014150504030F08D9158
:10C550000590801919F40020B9F7881B990B0895EC
:10C56000FB0155915523A9F0BF01DC014D91451701
:10C570004111E1F759F4CD010590002049F04D91AA
:10C5800040154111C9F3FB014111EFCF81E090E06B
:10C5900001970895FB01DC0102C001900D9241500A
:10C5A0005040D8F708956817790768F4FB01DC015B
:10C5B000E40FF51FA40FB51F02C002900E92415068
:10C5C0005040D8F708950C94CA62DC0101C06D9305
:10C5D00041505040E0F70895FB01DC010D90002030
:10C5E000E9F7119701900D920020E1F70895FC0101
:10C5F0008191861721F08823D9F7992708953197DB
:10C60000CF010895FB01DC018D910190801901108B
:10C61000D9F3990B0895FB01DC0101900D920020E4
:10C62000E1F70895FB01DC014150504030F08D915D
:10C630000190801919F40020B9F7881B990B08950F
:10C64000FB01DC014150504048F001900D92002068
:10C65000C9F701C01D9241505040E0F70895DC0138
:10C66000CB01FC01F999FECF06C0F2BDE1BDF89AFD
:10C67000319600B40D9241505040B8F70895A6E1AC
:10C68000B0E044E050E00C943163A8E1B0E042E057
:10C6900050E00C943163DC01A40FB51F41505040B1
:10C6A00048F0CB01840F951F2E910E945C6341508E
:10C6B0005040D0F70895262FF999FECF92BD81BD45
:10C6C000F89A019700B4021639F01FBA20BD0FB6D0
:10C6D000F894FA9AF99A0FBE08950396272F0E94AC
:10C6E0005C630E945B63252F0E945C63242F0C9483
:10C6F0005C630196272F0E945C630C945B63DC01F2
:10C70000CB0103C02D910E948A6341505040D0F765
:10C710000895262FF999FECF1FBA92BD81BD20BD85
:10C720000FB6F894FA9AF99A0FBE01960895242F3D
:10C730000E948A63252F0E948A630C949F630E9443
:0CC740008963272F0C948A63F894FFCFC4
:10C74C00020000000000C010000000000900010001
:10C75C000000460000000000000006010000000080
:10C76C00000900010000004600000000000000006D
:10C77C000000000000010000004600000000000066
:10C78C00000000000009000100000046000000004D
:10C79C00000000000000000900010000004600003D
:10C7AC00000000000000000000090001000000462D
:10C7BC0000000000000000907E000004020115CD76
:10C7CC005B07E5559A15B53B121F331349057007E6
:10C7DC009007B007D007E558DF58D958D358EB5815
:10C7EC00CD584758D9577057D75494540557995624
:10C7FC005656135687552C550001020203030303AA
:10C80C0004040404040404040505050505050505D4
:10C81C0005050505050505050606060606060606B4
:10C82C00060606060606060606060606060606069C
:10C83C000606060606060606070707070707070784
:10C84C00070707070707070707070707070707076C
:10C85C00070707070707070707070707070707075C
:10C86C00070707070707070707070707070707074C
:10C87C000707070707070707080808080808080834
:10C88C00080808080808080808080808080808081C
:10C89C00080808080808080808080808080808080C
:10C8AC0008080808080808080808080808080808FC
:10C8BC0008080808080808080808080808080808EC
:10C8CC0008080808080808080808080808080808DC
:10C8DC0008080808080808080808080808080808CC
:10C8EC0008080808080808080808080808080808BC
:08C8FC000808080808080808F4
:00000001FF
